:020000040000FA
:0408000098EF0BF072
:1008100003B275EF05F0F2B493EF05F09EB09BEFD5
:1008200005F09EB2A3EF05F0F2A81AEF04F0F2B2C1
:1008300023EF04F0F2B01FEF04F047EF0BF0F29655
:10084000F29047EF0BF0CD90F2929EA02DEF04F0C6
:100850000101533F2DEF04F0542BB2C1B6F1B3C1E7
:10086000B7F1B4C1B8F1B5C1B9F1AEC1B2F1AFC120
:10087000B3F1B0C1B4F1B1C1B5F1AAC1AEF1ABC130
:10088000AFF1ACC1B0F1ADC1B1F1A6C1AAF1A7C140
:10089000ABF1A8C1ACF1A9C1ADF1A2C1A6F1A3C150
:1008A000A7F1A4C1A8F1A5C1A9F19EC1A2F19FC160
:1008B000A3F1A0C1A4F1A1C1A5F19AC19EF19BC170
:1008C0009FF19CC1A0F19DC1A1F1CECF9AF1CFCFF4
:1008D0009BF153C19CF154C19DF1CF6ACE6A0101D5
:1008E000536B546B9E90CD800FBC0F8E0FBA7CEF74
:1008F00004F00F8A47EF0BF013880F8C0FBEB9EF8F
:1009000004F09AC19EF19BC19FF19CC1A0F19DC1D1
:10091000A1F19EC1A2F19FC1A3F1A0C1A4F1A1C107
:10092000A5F1A2C1A6F1A3C1A7F1A4C1A8F1A5C1D7
:10093000A9F1A6C1AAF1A7C1ABF1A8C1ACF1A9C1A7
:10094000ADF1AAC1AEF1ABC1AFF1ACC1B0F1ADC177
:10095000B1F1AEC1B2F1AFC1B3F1B0C1B4F1B1C147
:10096000B5F1B2C1B6F1B3C1B7F1B4C1B8F1B5C117
:10097000B9F101015E6B5F6B606B616B9A515E2731
:100980009B515F239C5160239D5161239E515E27A3
:100990009F515F23A0516023A1516123A2515E2783
:1009A000A3515F23A4516023A5516123A6515E2763
:1009B000A7515F23A8516023A9516123AA515E2743
:1009C000AB515F23AC516023AD516123AE515E2723
:1009D000AF515F23B0516023B1516123B2515E2703
:1009E000B3515F23B4516023B5516123B6515E27E3
:1009F000B7515F23B8516023B9516123D8900101E9
:100A0000613360335F335E33D8900101613360330B
:100A10005F335E33D8900101613360335F335E33FF
:100A200000C10CF101C10DF102C10EF103C10FF1C2
:100A300004C110F105C111F106C112F107C113F192
:100A400008C114F109C115F10AC116F10BC117F162
:100A500034C135F111B838EF05F00101620E046FB1
:100A6000010E056F000E066F000E076F41EF05F0D7
:100A70000101A70E046F020E056F000E066F000E37
:100A8000076F5EC100F15FC101F160C102F161C198
:100A900003F19FEC30F003BF04D01CBE02D01CA0B9
:100AA000108C11A059EF05F010BA59EF05F00F8026
:100AB000108A0CC100F10DC101F10EC102F10FC18C
:100AC00003F110C104F111C105F112C106F113C106
:100AD00007F114C108F115C109F116C10AF117C1D6
:100AE0000BF135C134F147EF0BF00392ABB2AB9889
:100AF000AB88030103EE00F080517F0BE92604C0B0
:100B0000EFFF802B8151805D700BD8A48B82000099
:100B10008051815D700BD8A48B9281518019D8B41B
:100B2000079047EF0BF0F2940101453F47EF0BF0C0
:100B3000462B47EF0BF09E900101533F47EF0BF020
:100B4000542B47EF0BF09E9211B843EF08F00400CE
:100B500066A1ABEF05F08BB4B5EF05F010ACB5EFC7
:100B600005F08B84109CB6EF05F08B94077C07ACE6
:100B7000D1EF05F0C274C2B4CBEF05F0C3CFB7F527
:100B8000C4CFB8F50501D890B833B733D890B8338F
:100B9000B733D2EF05F0C3CF55F1C4CF56F1D2EF42
:100BA00005F0C28207B444EF06F047C14BF148C1DB
:100BB0004CF149C14DF14AC14EF15EC162F15FC1D4
:100BC00063F160C164F161C165F113A8EAEF05F05A
:100BD000138C13989AC1BAF19BC1BBF19CC1BCF1B3
:100BE0009DC1BDF19EC1BEF19FC1BFF1A0C1C0F1C9
:100BF000A1C1C1F1A2C1C2F1A3C1C3F1A4C1C4F199
:100C0000A5C1C5F1A6C1C6F1A7C1C7F1A8C1C8F168
:100C1000A9C1C9F1AAC1CAF1ABC1CBF1ACC1CCF138
:100C2000ADC1CDF1AEC1CEF1AFC1CFF1B0C1D0F108
:100C3000B1C1D1F1B2C1D2F1B3C1D3F1B4C1D4F1D8
:100C4000B5C1D5F1B6C1D6F1B7C1D7F1B8C1D8F1A8
:100C5000B9C1D9F1B7C5B9F5B8C5BAF5B9C5BBF5CC
:100C6000BAC5BCF5010155515B2756515C23E86AB2
:100C70005D230E2E44EF06F05CC157F15DC158F1C3
:100C80005B6B5C6B5D6B078E0201002F47EF0BF017
:100C90003C0E006F1D50E00BE00AE86612881BBE98
:100CA00002D01BB4108E00C10CF101C10DF102C1C4
:100CB0000EF103C10FF104C110F105C111F106C11C
:100CC00012F107C113F108C114F109C115F10AC1EC
:100CD00016F10BC117F134C135F181AAACEF06F062
:100CE00015A4F7EF06F005012F51000AD8B43AEF2A
:100CF00007F005012F51010AD8B4B6EF06F005013F
:100D00002F51020AD8B4F7EF06F005012F51030A5C
:100D1000D8B4F7EF06F005012F51040AD8B4F7EF65
:100D200006F005012F51050AD8B4F7EF06F00501CA
:100D30002F51060AD8B4F7EF06F005012F51070A24
:100D4000D8B4F7EF06F005012F51320AD8B4B4EF4A
:100D500006F02F6B3AEF07F000011650030AD8B4E3
:100D6000F7EF06F03AEF07F03AEF07F005015767A3
:100D7000C1EF06F05867C1EF06F05967C1EF06F002
:100D80005A67C5EF06F03AEF07F05BC500F15CC5A6
:100D900001F15DC502F15EC503F10101010E046FB1
:100DA000000E056F000E066F000E076F9FEC30F00F
:100DB00000C15BF501C15CF502C15DF503C15EF5E3
:100DC00001010067EBEF06F00167EBEF06F0026749
:100DD000EBEF06F003673AEF07F057C55BF558C530
:100DE0005CF559C55DF55AC55EF524EF07F00FBEF9
:100DF0000CEF07F010A011EF07F00101476708EFB3
:100E000007F0486708EF07F0496708EF07F04A67FF
:100E10000CEF07F011EF07F007AE11EF07F024EF2A
:100E200007F00501312F3AEF07F03C0E316F302FFC
:100E30003AEF07F00101000E626FE00E636FA50E3E
:100E4000646F010E656F138800011650000AD8B454
:100E500032EF07F000011650030AD8B437EF07F05D
:100E60003AEF07F00001010E166E3AEF07F00001AD
:100E7000040E166E0501666B37B740EF07F066810A
:100E80000CC100F10DC101F10EC102F10FC103F15E
:100E900010C104F111C105F112C106F113C107F12E
:100EA00014C108F115C109F116C10AF117C10BF1FE
:100EB00035C134F100C10CF101C10DF102C10EF1D7
:100EC00003C10FF104C110F105C111F106C112F106
:100ED00007C113F108C114F109C115F10AC116F1D6
:100EE0000BC117F134C135F101018E677FEF07F0B7
:100EF0008F677FEF07F090677FEF07F0916783EFD1
:100F000007F0B4EF07F092C100F193C101F194C171
:100F100002F195C103F10101010E046F000E056F8E
:100F2000000E066F000E076F9FEC30F000C192F1CB
:100F300001C193F102C194F103C195F10101006770
:100F4000A9EF07F00167A9EF07F00267A9EF07F023
:100F50000367B4EF07F08EC192F18FC193F190C196
:100F600094F191C195F10F80D57ED5BE6ED0D6CFCC
:100F700047F1D7CF48F145C149F1E86AE8CF4AF1D6
:100F8000138A1CBE02D01CA0108C109047C100F127
:100F900048C101F149C102F14AC103F101010A0E40
:100FA000046F000E056F000E066F000E076F9FECBA
:100FB00030F003AF1080010154A7EBEF07F00F9A58
:100FC0000F9C0F9E0101000E5E6F600E5F6F3D0E65
:100FD000606F080E616F010147BFFBEF07F04867C4
:100FE000FBEF07F04967FBEF07F04A67FBEF07F0FD
:100FF000F28820EF08F0F2985E6B5F6B606B616BBC
:101000009A6B9B6B9C6B9D6B9E6B9F6BA06BA16B9C
:10101000A26BA36BA46BA56BA66BA76BA86BA96B4C
:10102000AA6BAB6BAC6BAD6BAE6BAF6BB06BB16BFC
:10103000B26BB36BB46BB56BB66BB76BB86BB96BAC
:10104000D76AD66A0101456B466B0CC100F10DC130
:1010500001F10EC102F10FC103F110C104F111C180
:1010600005F112C106F113C107F114C108F115C150
:1010700009F116C10AF117C10BF135C134F147EF7F
:101080000BF047EF0BF00201002FABEF0AF0D59EFB
:10109000D6CF47F1D7CF48F145C149F1E86AE8CF4B
:1010A0004AF1138AD76AD66A0101456B466BD58E21
:1010B0001D50E00BE00AE86612881BBE02D01BB48C
:1010C000108E1AAE1F8C00C10CF101C10DF102C1CE
:1010D0000EF103C10FF104C110F105C111F106C1F8
:1010E00012F107C113F108C114F109C115F10AC1C8
:1010F00016F10BC117F134C135F10FA0109A11B8D8
:101100008DEF08F00101620E046F010E056F000EF5
:10111000066F000E076F96EF08F00101A70E046F2F
:10112000020E056F000E066F000E076F47C100F13B
:1011300048C101F149C102F14AC103F19FEC30F00D
:1011400003BFA9EF08F01CBE02D01CA0108C11B088
:101150000F800CC100F10DC101F10EC102F10FC1F0
:1011600003F110C104F111C105F112C106F113C15F
:1011700007F114C108F115C109F116C10AF117C12F
:101180000BF135C134F102013C0E006F00C10CF1CE
:1011900001C10DF102C10EF103C10FF104C110F143
:1011A00005C111F106C112F107C113F108C114F113
:1011B00009C115F10AC116F10BC117F134C135F19E
:1011C00081BAE6EF08F015B225EF09F015A025EF7A
:1011D00009F015A470EF09F005012F51000AD8B4E9
:1011E000B3EF09F005012F51010AD8B42FEF09F030
:1011F00005012F51020AD8B470EF09F005012F51F3
:10120000030AD8B470EF09F005012F51040AD8B4CD
:1012100070EF09F005012F51050AD8B470EF09F0FD
:1012200005012F51060AD8B470EF09F005012F51BE
:10123000070AD8B470EF09F005012F51320AD8B46B
:101240002DEF09F02F6BB3EF09F000011650030AE0
:10125000D8B470EF09F0B3EF09F0B3EF09F005016E
:1012600057673AEF09F058673AEF09F059673AEFD4
:1012700009F05A673EEF09F0B3EF09F05BC500F1E2
:101280005CC501F15DC502F15EC503F10101010E0E
:10129000046F000E056F000E066F000E076F9FECC7
:1012A00030F000C15BF501C15CF502C15DF503C121
:1012B0005EF50101006764EF09F0016764EF09F072
:1012C000026764EF09F00367B3EF09F057C55BF5F8
:1012D00058C55CF559C55DF55AC55EF59DEF09F039
:1012E0000FBE85EF09F010A08AEF09F001014767F2
:1012F00081EF09F0486781EF09F0496781EF09F054
:101300004A6785EF09F08AEF09F007AE8AEF09F026
:101310009DEF09F00501312FB3EF09F03C0E316F5D
:10132000302FB3EF09F00101000E626FE00E636F22
:10133000A50E646F010E656F138800011650000A38
:10134000D8B4ABEF09F000011650030AD8B4B0EFDF
:1013500009F0B3EF09F00001010E166EB3EF09F0CA
:101360000001040E166E0501666B37B7B9EF09F080
:1013700066810CC100F10DC101F10EC102F10FC176
:1013800003F110C104F111C105F112C106F113C13D
:1013900007F114C108F115C109F116C10AF117C10D
:1013A0000BF135C134F100C10CF101C10DF102C1E5
:1013B0000EF103C10FF104C110F105C111F106C115
:1013C00012F107C113F108C114F109C115F10AC1E5
:1013D00016F10BC117F134C135F101018E67F8EF39
:1013E00009F08F67F8EF09F09067F8EF09F091675F
:1013F000FCEF09F02DEF0AF092C100F193C101F169
:1014000094C102F195C103F10101010E046F000EB8
:10141000056F000E066F000E076F9FEC30F000C1E5
:1014200092F101C193F102C194F103C195F101015F
:10143000006722EF0AF0016722EF0AF0026722EF4D
:101440000AF003672DEF0AF08EC192F18FC193F17C
:1014500090C194F191C195F10F80109047C100F1B6
:1014600048C101F149C102F14AC103F101010A0E6B
:10147000046F000E056F000E066F000E076F9FECE5
:1014800030F003AF1080010154A753EF0AF00F9A18
:101490000F9C0F9E0101000E5E6F600E5F6F3D0E90
:1014A000606F080E616F47C100F148C101F149C189
:1014B00002F14AC103F10101140E046F050E056F1C
:1014C000000E066F000E076F9FEC30F003AF6CEF5D
:1014D0000AF0F28891EF0AF0F2985E6B5F6B606B36
:1014E000616B9A6B9B6B9C6B9D6B9E6B9F6BA06BF8
:1014F000A16BA26BA36BA46BA56BA66BA76BA86B70
:10150000A96BAA6BAB6BAC6BAD6BAE6BAF6BB06B1F
:10151000B16BB26BB36BB46BB56BB66BB76BB86BCF
:10152000B96B0CC100F10DC101F10EC102F10FC187
:1015300003F110C104F111C105F112C106F113C18B
:1015400007F114C108F115C109F116C10AF117C15B
:101550000BF135C134F104008BB4B6EF0AF010ACD6
:10156000B6EF0AF08B84109CB7EF0AF08B94077CDF
:1015700007ACD2EF0AF0C274C2B4CCEF0AF0C3CF0A
:10158000B7F5C4CFB8F50501D890B833B733D890C4
:10159000B833B733D3EF0AF0C3CF55F1C4CF56F108
:1015A000D3EF0AF0C28207B445EF0BF047C14BF10D
:1015B00048C14CF149C14DF14AC14EF15EC162F1E1
:1015C0005FC163F160C164F161C165F113A8EBEF24
:1015D0000AF0138C13989AC1BAF19BC1BBF19CC15C
:1015E000BCF19DC1BDF19EC1BEF19FC1BFF1A0C1C3
:1015F000C0F1A1C1C1F1A2C1C2F1A3C1C3F1A4C193
:10160000C4F1A5C1C5F1A6C1C6F1A7C1C7F1A8C162
:10161000C8F1A9C1C9F1AAC1CAF1ABC1CBF1ACC132
:10162000CCF1ADC1CDF1AEC1CEF1AFC1CFF1B0C102
:10163000D0F1B1C1D1F1B2C1D2F1B3C1D3F1B4C1D2
:10164000D4F1B5C1D5F1B6C1D6F1B7C1D7F1B8C1A2
:10165000D8F1B9C1D9F1B7C5B9F5B8C5BAF5B9C5A9
:10166000BBF5BAC5BCF5010155515B2756515C234A
:10167000E86A5D230E2E45EF0BF05CC157F15DC1AA
:1016800058F15B6B5C6B5D6B078E47EF0BF002C034
:10169000E0FF005001C0D8FF1000A6B24DEF0BF0E4
:1016A0000CC0A9FF0BC0A8FFA69EA69CA684F29E14
:1016B000550EA76EAA0EA76EA682F28EA694A6B2AB
:1016C0005FEF0BF00C2A1200A96EA69EA69CA680C6
:1016D000A8500C2A120004012C0E826FA2EC0EF00E
:1016E000B4EC31F00C5064EC0BF0E8CF00F10C508E
:1016F00064EC0BF0E8CF01F101AF84EF0BF00101D6
:10170000FF0E026FFF0E036F3DEC31F0296790EF83
:101710000BF00401200E826FA2EC0EF095EF0BF09F
:1017200004012D0E826FA2EC0EF047EC2FF0120098
:1017300015941596076A0F6A106A116A126A136A7D
:10174000166A0F010D0EC16E860EC06E030EC26EBC
:101750000F01680E896E130E926E080E8A6EF30EDC
:10176000936E8B6A900E946EC80E64EC0BF0E8CF0B
:1017700025F000012550FE0AD8B4CAEF0BF0000195
:101780002550FD0AD8B4CFEF0BF00F0E266E8F0E4A
:10179000276E09D00E0E266E8E0E276E04D00D0E0B
:1017A000266E8D0E276E52EC32F092EC33F0F18EF5
:1017B000F19EFC0E64EC0BF0E8CF0BF00BA0118057
:1017C0000BA211820BA411840BA81188C90E64EC22
:1017D0000BF0E8CF1AF0CA0E64EC0BF0E8CF1BF068
:1017E000CB0E64EC0BF0E8CF1CF0CC0E64EC0BF0ED
:1017F000E8CF1DF0FB0E64EC0BF0E8CF38F0CE0E16
:1018000064EC0BF0E8CF14F0CD0E64EC0BF0E8CFF5
:1018100037F01F6A206A0E6A01015B6B5C6B5D6BBF
:10182000576B586BF29A0101476B486B496B4A6BD7
:101830004B6B4C6B4D6B4E6B4F6B506B516B526BDC
:10184000456B466BD76AD66A0F01280ED56EF28AB1
:101850009D90B00ECD6E01015E6B5F6B606B616B36
:10186000626B636B646B656B666B676B686B696BF4
:10187000536B546BCF6ACE6A0F9A0F9C0F9E9D805C
:10188000760ECA6E9D8202013C0E006FCC6A160E67
:1018900064EC0BF0E8CF00F1170E64EC0BF0E8CF2E
:1018A00001F1180E64EC0BF0E8CF02F1190E64ECB4
:1018B0000BF0E8CF03F1010103AF79EF0CF0B4ECCA
:1018C00031F0160E0C6E00C10BF04DEC0BF0170E44
:1018D0000C6E01C10BF04DEC0BF0180E0C6E02C13A
:1018E0000BF04DEC0BF0190E0C6E03C10BF04DEC30
:1018F0000BF000C18EF101C18FF102C190F103C163
:1019000091F100C192F101C193F102C194F103C1BF
:1019100095F11A0E64EC0BF0E8CF00F11B0E64ECAD
:101920000BF0E8CF01F11C0E64EC0BF0E8CF02F1F4
:101930001D0E64EC0BF0E8CF03F1010103AFCFEF14
:101940000CF0B4EC31F01A0E0C6E00C10BF04DEC43
:101950000BF01B0E0C6E01C10BF04DEC0BF01C0ECE
:101960000C6E02C10BF04DEC0BF01D0E0C6E03C1A2
:101970000BF04DEC0BF01A0E64EC0BF0E8CF00F11D
:101980001B0E64EC0BF0E8CF01F11C0E64EC0BF0C5
:10199000E8CF02F11D0E64EC0BF0E8CF03F100C1BB
:1019A00096F101C197F102C198F103C199F1240E9A
:1019B000AC6E900EAB6E240EAC6E080EB86E000EC0
:1019C000B06E1F0EAF6E0401806B816B0F01900E25
:1019D000AB6E0F019D8A0301806B816BC26B8B9292
:1019E00023EC37F023EC37F005EC39F001EC35F05F
:1019F000200E64EC0BF0E8CF2FF505012F51FF0A04
:101A0000D8A40AEF0DF02F6B200E0C6E2FC50BF033
:101A10004DEC0BF00501010E306F3C0E316F250EC1
:101A200064EC0BF0E8CF00F1260E64EC0BF0E8CF8D
:101A300001F1270E64EC0BF0E8CF02F1280E64EC04
:101A40000BF0E8CF03F1010103AF41EF0DF0B4EC6F
:101A500031F0250E0C6E00C10BF04DEC0BF0260E94
:101A60000C6E01C10BF04DEC0BF0270E0C6E02C199
:101A70000BF04DEC0BF0280E0C6E03C10BF04DEC8F
:101A80000BF000C157F501C158F502C159F503C16A
:101A90005AF500C15BF501C15CF502C15DF503C1FA
:101AA0005EF5290E64EC0BF0E8CF5FF5050160519F
:101AB0005F5DD8A05FC560F5210E64EC0BF0E8CF48
:101AC00000F1220E64EC0BF0E8CF01F1230E64EC80
:101AD0000BF0E8CF02F1240E64EC0BF0E8CF03F139
:101AE000010103AFA2EF0DF0B4EC31F0210E0C6E4A
:101AF00000C10BF04DEC0BF0220E0C6E01C10BF08F
:101B00004DEC0BF0230E0C6E02C10BF04DEC0BF004
:101B1000240E0C6E03C10BF04DEC0BF0210E64ECA7
:101B20000BF0E8CF00F1220E64EC0BF0E8CF01F1EE
:101B3000230E64EC0BF0E8CF02F1240E64EC0BF002
:101B4000E8CF03F100C161F501C162F502C163F59F
:101B500003C164F512EC34F02FEC33F065EC32F095
:101B60001590C70E64EC0BF0E8CF00F1010100B155
:101B7000BDEF0DF01592BEEF0DF0158281AACCEFEE
:101B80000DF015B4C7EF0DF01580CCEF0DF044EC5F
:101B900039F015A0ADEF39F007900001F28EF28C0C
:101BA00012AE03D012BC7AEF19F007B0C6EF2DF0D9
:101BB0000FB0B6EF26F010BEB6EF26F012B8B6EFB3
:101BC00026F000011650010AD8B4BEEF1DF081BA0C
:101BD000F2EF0DF000011650040AD8B437EF1CF0F4
:101BE000F8EF0DF000011650040AD8B4FAEF1DF01A
:101BF0000301805181197F0BD8B4C6EF2DF013EE8D
:101C000000F081517F0BE126812BE7CFE8FFE00B4D
:101C1000D8B4C6EF2DF023EE82F0C2513F0BD92687
:101C2000E7CFDFFFC22BDF50780AD8A4C6EF2DF034
:101C3000078092C100F193C101F194C102F195C1F5
:101C400003F10101040E046F000E056F000E066F14
:101C5000000E076F9FEC30F000AF38EF0EF001017F
:101C6000030E926F000E936F000E946F000E956F2F
:101C700003018251720AD8B437EF26F08251520A1A
:101C8000D8B437EF26F08251750AD8B437EF26F072
:101C90008251680AD8B4B6EF0EF08251630AD8B404
:101CA00080EF2AF08251690AD8B404EF21F0825102
:101CB0007A0AD8B417EF22F08251490AD8B4A3EFB8
:101CC00020F08251500AD8B4C1EF1FF08251700A3F
:101CD000D8B404EF20F08251540AD8B42FEF20F08A
:101CE0008251740AD8B475EF20F08251410AD8B4F9
:101CF000BBEF0FF082514B0AD8B4B8EF0EF082510F
:101D00006D0AD8B42BEF14F082514D0AD8B444EFC9
:101D100014F08251730AD8B467EF25F08251530A48
:101D2000D8B4CCEF25F082514C0AD8B4D3EF14F0DC
:101D30008251590AD8B47CEF13F012AE01D0128C44
:101D4000B7EF2AF0040114EE00F080517F0BE1267A
:101D500082C4E7FF802B120004010D0E826FA2ECFB
:101D60000EF00A0E826FA2EC0EF01200B5EF2AF010
:101D700004014B0E826FA2EC0EF004012C0E826F58
:101D8000A2EC0EF081B802D037B630D003018351F7
:101D9000430AD8B4FDEF0EF003018351630AD8B4AF
:101DA000FFEF0EF003018351520AD8B401EF0FF098
:101DB00003018351720AD8B403EF0FF0030183517A
:101DC000470AD8B405EF0FF003018351670AD8B46E
:101DD00007EF0FF003018351540AD8B409EF0FF055
:101DE00003018351740AD8B479EF0FF003018351D2
:101DF000550AD8B40BEF0FF083D037807BD03790E3
:101E000079D0378277D0379275D0378473D03794B2
:101E100071D037866FD084C330F185C331F186C36A
:101E200032F187C333F10101296B02EC32F079EC16
:101E300031F000C104F101C105F102C106F103C195
:101E400007F1F5EC31F0200EF86EF76AF66A09003A
:101E5000F5CF2CF10900F5CF2DF10900F5CF2EF1CA
:101E60000900F5CF2FF10900F5CF30F10900F5CFCA
:101E700031F10900F5CF32F10900F5CF33F101015D
:101E8000296B02EC32F079EC31F09FEC30F001017B
:101E9000006752EF0FF0016752EF0FF0026752EF49
:101EA0000FF0036701D025D004014E0E826FA2EC23
:101EB0000EF004016F0E826FA2EC0EF004014D0EC5
:101EC000826FA2EC0EF00401610E826FA2EC0EF0A4
:101ED0000401740E826FA2EC0EF00401630E826F97
:101EE000A2EC0EF00401680E826FA2EC0EF0B5EFCA
:101EF0002AF03796CD0E0C6E37C00BF04DEC0BF080
:101F0000CD0E64EC0BF0E8CF37F037B006D004010B
:101F1000630E826FA2EC0EF005D00401430E826FB7
:101F2000A2EC0EF037B206D00401720E826FA2EC62
:101F30000EF005D00401520E826FA2EC0EF037B401
:101F400006D00401670E826FA2EC0EF005D00401EA
:101F5000470E826FA2EC0EF037B606D00401740E65
:101F6000826FA2EC0EF005D00401540E826FA2EC39
:101F70000EF0B5EF2AF00401410E826FA2EC0EF0D4
:101F800003018351310AD8B49CEF12F0030183514D
:101F9000320AD8B4CCEF11F003018351330AD8B41C
:101FA00055EF11F003018351340AD8B445EF10F016
:101FB00003018351350AD8B4E5EF0FF004013F0E59
:101FC000826FA2EC0EF0B5EF2AF003018451300AC3
:101FD000D8B40BEF10F003018451310AD8B40EEFDE
:101FE00010F003018451650AD8B4FFEF0FF003012C
:101FF0008451640AD8B402EF10F00FEF10F038905B
:1020000003EF10F03880FB0E0C6E38C00BF04DEC77
:102010000BF00FEF10F08B900FEF10F08B8004019E
:10202000350E826FA2EC0EF004012C0E826FA2EC32
:102030000EF08BB023EF10F00401300E826FA2EC93
:102040000EF028EF10F00401310E826FA2EC0EF0BA
:1020500004012C0E826FA2EC0EF0FB0E64EC0BF070
:10206000E8CF38F038A03CEF10F00401640E826F26
:10207000A2EC0EF041EF10F00401650E826FA2ECAD
:102080000EF043EF10F0B5EF2AF0CC0E64EC0BF03D
:10209000E8CF0BF004012C0E826FA2EC0EF00301CE
:1020A0008451310AD8B469EF10F003018451300A29
:1020B000D8B46BEF10F0030184514D0AD8B475EF1A
:1020C00010F003018451540AD8B47CEF10F093EF60
:1020D00010F08A8401D08A940BAE04D00BAC02D0ED
:1020E0000BBA21D0E00E0B1218D01F0E0B1685393B
:1020F000E844E00B0B1211D0E00E0B16F5EC31F0BA
:1021000085C332F186C333F10101296B02EC32F051
:1021100079EC31F000511F0B0B12CC0E0C6E0BC082
:102120000BF04DEC0BF00401340E826FA2EC0EF0BC
:1021300004012C0E826FA2EC0EF0CC0E64EC0BF0BE
:10214000E8CF1DF08AB406D00401300E826FA2ECF5
:102150000EF005D00401310E826FA2EC0EF00401E6
:102160002C0E826FA2EC0EF01D38E840070BE8CF72
:1021700082F40401300E8227A2EC0EF004012C0E32
:10218000826FA2EC0EF0B4EC31F01D501F0BE8CFC3
:1021900000F13DEC31F032C182F40401300E8227AF
:1021A000A2EC0EF033C182F40401300E8227A2ECBF
:1021B0000EF004012C0E826FA2EC0EF0B4EC31F0A4
:1021C00031C000F100AF0BD0FF0E016FFF0E026FA8
:1021D000FF0E036F04012D0E826FA2EC0EF03DEC9A
:1021E00031F031C182F40401300E8227A2EC0EF0EE
:1021F00032C182F40401300E8227A2EC0EF033C10A
:1022000082F40401300E8227A2EC0EF004012C0EA1
:10221000826FA2EC0EF0B4EC31F030C000F13DEC76
:1022200031F031C182F40401300E8227A2EC0EF0AD
:1022300032C182F40401300E8227A2EC0EF033C1C9
:1022400082F40401300E8227A2EC0EF004012C0E61
:10225000826FA2EC0EF0B4EC31F032C000F100AFAE
:102260000BD0FF0E016FFF0E026FFF0E036F040114
:102270002D0E826FA2EC0EF03DEC31F031C182F4F4
:102280000401300E8227A2EC0EF032C182F4040168
:10229000300E8227A2EC0EF033C182F40401300E1E
:1022A0008227A2EC0EF0B5EF2AF0CB0E64EC0BF017
:1022B000E8CF0BF004012C0E826FA2EC0EF00301AC
:1022C0008451450AD8B479EF11F003018451440ACE
:1022D000D8B47CEF11F003018451300AD8B47FEFF9
:1022E00011F003018451310AD8B483EF11F08EEF5D
:1022F00011F00B9E88EF11F00B8E88EF11F0FC0EA1
:102300000B1688EF11F0FC0E0B160B8088EF11F006
:10231000CB0E0C6E0BC00BF04DEC0BF00401330E2A
:10232000826FA2EC0EF004012C0E826FA2EC0EF074
:10233000CB0E64EC0BF0E8CF1CF01CBEA7EF11F045
:102340000401450E826FA2EC0EF0ACEF11F0040117
:10235000440E826FA2EC0EF004012C0E826FA2ECF0
:102360000EF00401300E826FA2EC0EF004012C0E70
:10237000826FA2EC0EF01CB0C5EF11F00401300E1C
:10238000826FA2EC0EF0CAEF11F00401310E826FE1
:10239000A2EC0EF0B5EF2AF0CA0E64EC0BF0E8CF19
:1023A0000BF004012C0E826FA2EC0EF0030184519D
:1023B000450AD8B408EF12F003018451440AD8B496
:1023C0000BEF12F0030184514D0AD8B414EF12F050
:1023D00003018451410AD8B40EEF12F00301845175
:1023E000460AD8B411EF12F003018451560AD8B44A
:1023F0001CEF12F003018451500AD8B427EF12F0F9
:1024000003018451520AD8B42AEF12F033EF12F0CC
:102410000B9E2DEF12F00B8E2DEF12F00B9C2DEF7B
:1024200012F00B8C2DEF12F0FC0E0B1685C3E8FF9B
:10243000030B0B122DEF12F0C70E0B1685C3E8FF2E
:10244000070BE846E846E8460B122DEF12F00B8426
:102450002DEF12F00B942DEF12F0CA0E0C6E0BC084
:102460000BF04DEC0BF0CA0E64EC0BF0E8CF1BF058
:102470000401320E826FA2EC0EF004012C0E826F6A
:10248000A2EC0EF01BBE4CEF12F00401450E826F61
:10249000A2EC0EF051EF12F00401440E826FA2EC98
:1024A0000EF004012C0E826FA2EC0EF01BC0E8FFB0
:1024B000030BE8CF82F40401300E8227A2EC0EF069
:1024C00004012C0E826FA2EC0EF01BBC6FEF12F019
:1024D0000401410E826FA2EC0EF074EF12F00401C1
:1024E000460E826FA2EC0EF004012C0E826FA2EC5D
:1024F0000EF01BC0E8FF380BE842E842E842E8CFA4
:1025000082F40401300E8227A2EC0EF004012C0E9E
:10251000826FA2EC0EF01BB495EF12F00401520E84
:10252000826FA2EC0EF09AEF12F00401500E826F4F
:10253000A2EC0EF0B5EF2AF0C90E64EC0BF0E8CF78
:102540000BF004012C0E826FA2EC0EF003018451FB
:10255000450AD8B4BAEF12F003018451440AD8B442
:10256000BDEF12F0030184514D0AD8B4C0EF12F050
:10257000CEEF12F00B9EC8EF12F00B8EC8EF12F0E8
:10258000F80E0B1685C3E8FF070B0B12C8EF12F00D
:10259000C90E0C6E0BC00BF04DEC0BF00401310EAC
:1025A000826FA2EC0EF004012C0E826FA2EC0EF0F2
:1025B000C90E64EC0BF0E8CF1AF01ABE06D0040185
:1025C000450E826FA2EC0EF005D00401440E826F1E
:1025D000A2EC0EF004012C0E826FA2EC0EF01AC0D9
:1025E000E8FF070BE8CF82F40401300E8227A2EC4B
:1025F0000EF004012C0E826FA2EC0EF00780B4ECFA
:1026000031F02CC0E8FF003B00430043030B3DECDE
:1026100031F033C182F40401300E8227A2EC0EF0B7
:1026200004012C0E826FA2EC0EF0B4EC31F02CC041
:1026300001F1019F019D2DC000F101013DEC31F040
:102640002FC182F40401300E8227A2EC0EF030C1BB
:1026500082F40401300E8227A2EC0EF031C182F424
:102660000401300E8227A2EC0EF032C182F4040184
:10267000300E8227A2EC0EF033C182F40401300E3A
:102680008227A2EC0EF004012C0E826FA2EC0EF059
:10269000B4EC31F02EC001F12FC000F1D89001331D
:1026A0000033D8900133003301013DEC31F02FC1EC
:1026B00082F40401300E8227A2EC0EF030C182F4C5
:1026C0000401300E8227A2EC0EF031C182F4040125
:1026D000300E8227A2EC0EF032C182F40401300EDB
:1026E0008227A2EC0EF033C182F40401300E82275F
:1026F000A2EC0EF0B5EF2AF0FC0E64EC0BF0E8CF84
:102700000BF003018351520AD8B4B3EF13F0030165
:102710008351720AD8B4B6EF13F003018351500A03
:10272000D8B4B9EF13F003018351700AD8B4BCEFE9
:1027300013F003018351550AD8B4BFEF13F003011E
:102740008351750AD8B4C2EF13F003018351430AD1
:10275000D8B4CBEF13F003018351630AD8B4CEEFA2
:1027600013F0D7EF13F00B90D1EF13F00B80D1EFF4
:1027700013F00B92D1EF13F00B82D1EF13F00B9407
:10278000D1EF13F00B84D1EF13F00B96D1EF13F0D0
:102790000B86D1EF13F00B98D1EF13F00B88D1EF2C
:1027A00013F0FC0E0C6E0BC00BF04DEC0BF00401A3
:1027B000590E826FA2EC0EF01190119211941198A3
:1027C000FC0E64EC0BF0E8CF0BF00BA011800BA219
:1027D00011820BA411840BA8118811A0F7EF13F03C
:1027E0000401520E826FA2EC0EF0FCEF13F0040114
:1027F000720E826FA2EC0EF011A806EF14F0040125
:10280000430E826FA2EC0EF00BEF14F00401630E86
:10281000826FA2EC0EF011A215EF14F00401500E1D
:10282000826FA2EC0EF01AEF14F00401700E826FAA
:10283000A2EC0EF011A424EF14F00401550E826FE7
:10284000A2EC0EF029EF14F00401750E826FA2ECD9
:102850000EF0B5EF2AF004016D0E826FA2EC0EF0BF
:1028600003018351300AD8B483EF14F0030183517C
:10287000310AD8B496EF14F003018351320AD8B468
:10288000A9EF14F0B7EF2AF004014D0E826FA2EC0D
:102890000EF0F5EC31F084C331F185C332F186C31B
:1028A00033F10101296B02EC32F079EC31F00301D4
:1028B0008351300AD8B46BEF14F003018351310A0D
:1028C000D8B473EF14F003018351320AD8B47BEF0C
:1028D00014F0B7EF2AF0FD0E0C6E00C10BF04DECBA
:1028E0000BF083EF14F0FE0E0C6E00C10BF04DECFC
:1028F0000BF096EF14F0FF0E0C6E00C10BF04DECD8
:102900000BF0A9EF14F00401300E826FA2EC0EF070
:1029100004012C0E826FA2EC0EF0B4EC31F0FD0E2F
:1029200064EC0BF0E8CF00F1BAEF14F00401310EC3
:10293000826FA2EC0EF004012C0E826FA2EC0EF05E
:10294000B4EC31F0FE0E64EC0BF0E8CF00F1BAEF1E
:1029500014F00401320E826FA2EC0EF0B4EC31F0F0
:1029600004012C0E826FA2EC0EF0FF0E64EC0BF053
:10297000E8CF00F13DEC31F031C182F40401300EBA
:102980008227A2EC0EF032C182F40401300E8227BD
:10299000A2EC0EF033C182F40401300E8227A2ECC7
:1029A0000EF0B5EF2AF003018351300AD8B427EFB7
:1029B0001AF003018351310AD8B465EF1BF003010B
:1029C0008351320AD8B4D3EF1BF003018351330A89
:1029D000D8B4E3EF1BF003018351340AD8B43EEFBF
:1029E0001CF003018351350AD8B412EF1EF0030125
:1029F0008351360AD8B440EF1EF003018351370AE1
:102A0000D8B4FFEF17F003018351380AD8B49DEF13
:102A100018F003018351440AD8B42BEF16F00301D8
:102A20008351640AD8B44BEF16F003018351460A70
:102A3000D8B417EF1DF0030183514D0AD8B478EFD5
:102A400016F0030183516D0AD8B492EF16F003011A
:102A500083515A0AD8B4DFEF1AF003018351490AAF
:102A6000D8B440EF1FF003018351500AD8B472EF7D
:102A70001EF003018351540AD8B4EBEF1EF003019A
:102A80008351630AD8B4B2EF16F003018351430AAD
:102A9000D8B4AAEF17F003018351730AD8B4B0EF8A
:102AA00016F003018351610AD8B478EF15F00301E1
:102AB0008351650AD8B477EF1AF003018351450AB0
:102AC000D8B485EF1AF003018351620AD8B493EFAA
:102AD0001AF003018351420AD8B4A1EF1AF003019E
:102AE0008351760AD8B4AFEF1AF0D8A4B7EF2AF022
:102AF00004014C0E826FA2EC0EF00401610E826F95
:102B0000A2EC0EF02FEC33F004012C0E826FA2EC3D
:102B10000EF0B4EC31F0AFC500F101013DEC31F045
:102B200031C182F40401300E8227A2EC0EF032C1D2
:102B300082F40401300E8227A2EC0EF033C182F43D
:102B40000401300E8227A2EC0EF004012C0E826FDD
:102B5000A2EC0EF0B4EC31F0B0C500F101013DEC97
:102B600031F031C182F40401300E8227A2EC0EF064
:102B700032C182F40401300E8227A2EC0EF033C180
:102B800082F40401300E8227A2EC0EF004012C0E18
:102B9000826FA2EC0EF0B4EC31F0B1C500F101018E
:102BA0003DEC31F031C182F40401300E8227A2ECF9
:102BB0000EF032C182F40401300E8227A2EC0EF036
:102BC00033C182F40401300E8227A2EC0EF004011E
:102BD0002C0E826FA2EC0EF0B4EC31F0B2C500F115
:102BE00001013DEC31F031C182F40401300E822745
:102BF000A2EC0EF032C182F40401300E8227A2EC66
:102C00000EF033C182F40401300E8227A2EC0EF0E4
:102C100004012C0E826FA2EC0EF0B4EC31F0B6C5BC
:102C200000F101013DEC31F031C182F40401300EBC
:102C30008227A2EC0EF032C182F40401300E82270A
:102C4000A2EC0EF033C182F40401300E8227A2EC14
:102C50000EF06EEF1EF003018451300AD8B437EF46
:102C600016F003018451310AD8B43BEF16F01592E7
:102C700015963CEF16F01582C70E64EC0BF0E8CF0A
:102C800000F10101008115A20091C70E0C6E00C178
:102C90000BF04DEC0BF0C70E64EC0BF0E8CF00F13D
:102CA000010100B157EF16F0159258EF16F015829A
:102CB00004014C0E826FA2EC0EF00401640E826FD0
:102CC000A2EC0EF004012C0E826FA2EC0EF015B2F5
:102CD00071EF16F00401300E826FA2EC0EF076EF69
:102CE00016F00401310E826FA2EC0EF0B5EF2AF05F
:102CF000F5EC31F084C333F102EC32F079EC31F0D1
:102D0000200E0C6E00C10BF04DEC0BF000C12FF546
:102D100005012F51000A06E005012F51010A02E0CA
:102D200092EC33F004014C0E826FA2EC0EF0040121
:102D30004D0E826FA2EC0EF004012C0E826FA2ECFD
:102D40000EF0B4EC31F02FC500F13DEC31F033C1A1
:102D500082F40401300E8227A2EC0EF06EEF1EF01A
:102D6000ADEF39F004014C0E826FA2EC0EF00401BD
:102D7000630E826FA2EC0EF065EC32F004012C0EB3
:102D8000826FA2EC0EF0C7EC16F06EEF1EF0B4EC02
:102D900031F0B5C500F10101003B0F0E00173DEC0D
:102DA00031F033C182F40401300E8227A2EC0EF020
:102DB000B5C500F101010F0E010100173DEC31F026
:102DC00033C182F40401300E8227A2EC0EF004011C
:102DD0002D0E826FA2EC0EF0B4C500F10101003B94
:102DE0000F0E00173DEC31F033C182F40401300EB8
:102DF0008227A2EC0EF0B4C500F101010F0E010113
:102E000000173DEC31F033C182F40401300E82270B
:102E1000A2EC0EF004012D0E826FA2EC0EF0B3C5F1
:102E200000F10101003B0F0E00173DEC31F033C102
:102E300082F40401300E8227A2EC0EF0B3C500F13B
:102E400001010F0E010100173DEC31F033C182F496
:102E50000401300E8227A2EC0EF00401200E826FD6
:102E6000A2EC0EF0B2C500F10F0E010100173DEC0F
:102E700031F033C182F40401300E8227A2EC0EF04F
:102E80000401200E826FA2EC0EF0B1C500F1010129
:102E90000101003B0F0E00173DEC31F033C182F40D
:102EA0000401300E8227A2EC0EF0B1C500F1010141
:102EB0000F0E010100173DEC31F033C182F4040123
:102EC000300E8227A2EC0EF004013A0E826FA2ECC3
:102ED0000EF0B0C500F10101003B0F0E00173DECF4
:102EE00031F033C182F40401300E8227A2EC0EF0DF
:102EF000B0C500F101010F0E010100173DEC31F0EA
:102F000033C182F40401300E8227A2EC0EF00401DA
:102F10003A0E826FA2EC0EF0AFC500F10101003B4A
:102F20000F0E00173DEC31F033C182F40401300E76
:102F30008227A2EC0EF0AFC500F101010F0E0017C1
:102F40003DEC31F033C182F40401300E8227A2EC53
:102F50000EF0120084C3E8FF0F0BE83AE8CFB5F596
:102F600085C3E8FF0F0B0501B51387C3E8FF0F0BFF
:102F7000E83AE8CFB4F588C3E8FF0F0B0501B413B6
:102F80008AC3E8FF0F0BE83AE8CFB3F58BC3E8FF3D
:102F90000F0B0501B3138DC3E8FF0F0BE8CFB2F59C
:102FA0008FC3E8FF0F0BE83AE8CFB1F590C3E8FF15
:102FB0000F0B0501B11392C3E8FF0F0BE83AE8CFFE
:102FC000B0F593C3E8FF0F0B0501B01395C3E8FFFD
:102FD0000F0BE83AE8CFAFF596C3E8FF0F0B0501FA
:102FE000AF13D1EC32F004014C0E826FA2EC0EF064
:102FF0000401430E826FA2EC0EF0BCEF16F00784C2
:1030000004014C0E826FA2EC0EF00401370E826FA9
:10301000A2EC0EF004012C0E826FA2EC0EF0050162
:103020002E51130A06E005012E51170A0DE09AEF02
:1030300018F00101000E006F000E016F100E026FFC
:10304000000E036F2DEF18F00101000E006F000E4F
:10305000016F000E026F010E036F3DEC31F02AC1CB
:1030600082F40401300E8227A2EC0EF02BC182F410
:103070000401300E8227A2EC0EF02CC182F4040170
:10308000300E8227A2EC0EF02DC182F40401300E26
:103090008227A2EC0EF02EC182F40401300E8227AA
:1030A000A2EC0EF02FC182F40401300E8227A2ECB4
:1030B0000EF030C182F40401300E8227A2EC0EF033
:1030C00031C182F40401300E8227A2EC0EF032C12D
:1030D00082F40401300E8227A2EC0EF033C182F498
:1030E0000401300E8227A2EC0EF004012C0E826F38
:1030F000A2EC0EF00101100E006F000E016F000E29
:10310000026F000E036F3DEC31F031C182F4040117
:10311000300E8227A2EC0EF032C182F40401300E90
:103120008227A2EC0EF033C182F40401300E822714
:10313000A2EC0EF007946EEF1EF00501216B226BDE
:10314000236B246B04014C0E826FA2EC0EF0040181
:10315000380E826FA2EC0EF004012C0E826FA2ECEE
:103160000EF00101100E006F000E016F000E026FD5
:10317000000E036F3DEC31F02AC182F40401300EE1
:103180008227A2EC0EF02BC182F40401300E8227BC
:10319000A2EC0EF02CC182F40401300E8227A2ECC6
:1031A0000EF02DC182F40401300E8227A2EC0EF045
:1031B0002EC182F40401300E8227A2EC0EF02FC142
:1031C00082F40401300E8227A2EC0EF030C182F4AA
:1031D0000401300E8227A2EC0EF031C182F404010A
:1031E000300E8227A2EC0EF032C182F40401300EC0
:1031F0008227A2EC0EF033C182F40401300E822744
:10320000A2EC0EF004012C0E826FA2EC0EF025C58C
:1032100000F126C501F127C502F128C503F101011E
:10322000100E046F000E056F000E066F000E076F84
:10323000D0EC30F000C133F501C134F502C135F5F1
:1032400003C136F53DEC31F02AC182F40401300EA1
:103250008227A2EC0EF02BC182F40401300E8227EB
:10326000A2EC0EF02CC182F40401300E8227A2ECF5
:103270000EF02DC182F40401300E8227A2EC0EF074
:103280002EC182F40401300E8227A2EC0EF02FC171
:1032900082F40401300E8227A2EC0EF030C182F4D9
:1032A0000401300E8227A2EC0EF031C182F4040139
:1032B000300E8227A2EC0EF032C182F40401300EEF
:1032C0008227A2EC0EF033C182F40401300E822773
:1032D000A2EC0EF0ACEC0EF00501336777EF19F0BD
:1032E000346777EF19F0356777EF19F0366702D05A
:1032F00016EF1AF0129E129C21C500F122C501F1B1
:1033000023C502F124C503F1899A400EC76E200E31
:10331000C66E9E96C69E0B0EC96EFF0E9EB602D05E
:10332000E82EFCD79E96C69E02C1C9FFFF0E9EB630
:1033300002D0E82EFCD79E96C69E01C1C9FFFF0EA3
:103340009EB602D0E82EFCD79E96C69E00C1C9FF4D
:10335000FF0E9EB602D0E82EFCD79E96C69EC9529E
:10336000FF0E9EB602D0E82EFCD70501100E326F7C
:10337000040114EE00F080517F0BE1269E96C69E5C
:10338000C952FF0E9EB602D0E82EFCD7C9CFE7FF88
:103390000401802B0501322FB8EF19F0898A33C55B
:1033A00000F134C501F135C502F136C503F1010163
:1033B000010E046F000E056F000E066F000E076F02
:1033C0009FEC30F000C133F501C134F502C135F591
:1033D00003C136F505013367F5EF19F03467F5EFF2
:1033E00019F03567F5EF19F0366702D016EF1AF0CD
:1033F00021C500F122C501F123C502F124C503F165
:103400000101100E046F000E056F000E066F000E16
:10341000076FA4EC30F000C121F501C122F502C113
:1034200023F503C124F5128EB7EF2AF00401450EEF
:10343000826FA2EC0EF004014F0E826FA2EC0EF030
:103440000401460E826FA2EC0EF06EEF1EF00784B0
:1034500005EC39F0B4EC31F02DC500F13DEC31F064
:1034600004014C0E826FA2EC0EF00401300E826F4C
:10347000A2EC0EF004012C0E826FA2EC0EF031C112
:1034800082F40401300E8227A2EC0EF032C182F4E5
:103490000401300E8227A2EC0EF033C182F4040145
:1034A000300E8227A2EC0EF004012C0E826FA2ECEB
:1034B0000EF0B4EC31F02EC500F13DEC31F031C12D
:1034C00082F40401300E8227A2EC0EF032C182F4A5
:1034D0000401300E8227A2EC0EF033C182F4040105
:1034E000300E8227A2EC0EF007946EEF1EF004015E
:1034F0004C0E826FA2EC0EF00401650E826FA2ECFE
:103500000EF0A5EC34F06EEF1EF004014C0E826F4D
:10351000A2EC0EF00401450E826FA2EC0EF0BCECA2
:1035200034F06EEF1EF004014C0E826FA2EC0EF030
:103530000401620E826FA2EC0EF0EAEC34F06EEF42
:103540001EF004014C0E826FA2EC0EF00401420E3C
:10355000826FA2EC0EF0D3EC34F06EEF1EF004019B
:103560004C0E826FA2EC0EF00401760E826FA2EC7C
:103570000EF004012C0E826FA2EC0EF0000125501B
:10358000FE0AD8B4D1EF1AF000012550FD0AD8B4D4
:10359000D8EF1AF00401300E826FA2EC0EF06EEF3D
:1035A0001EF00401310E826FA2EC0EF06EEF1EF0E1
:1035B0000401320E826FA2EC0EF06EEF1EF00401D9
:1035C0004C0E826FA2EC0EF004015A0E826FA2EC38
:1035D0000EF004012C0E826FA2EC0EF005EC39F017
:1035E000B4EC31F005012E51130A06E005012E510D
:1035F000170A0DE010EF1BF00101000E006F000E26
:10360000016F100E026F000E036F10EF1BF001012F
:10361000000E006F000E016F000E026F010E036FAF
:103620000101100E046F000E056F000E066F000EF4
:10363000076FD0EC30F03DEC31F02AC182F4040188
:10364000300E8227A2EC0EF02BC182F40401300E62
:103650008227A2EC0EF02CC182F40401300E8227E6
:10366000A2EC0EF02DC182F40401300E8227A2ECF0
:103670000EF02EC182F40401300E8227A2EC0EF06F
:103680002FC182F40401300E8227A2EC0EF030C16B
:1036900082F40401300E8227A2EC0EF031C182F4D4
:1036A0000401300E8227A2EC0EF032C182F4040134
:1036B000300E8227A2EC0EF033C182F40401300EEA
:1036C0008227A2EC0EF06EEF1EF0078404014C0E70
:1036D000826FA2EC0EF00401310E826FA2EC0EF0AC
:1036E00004012C0E826FA2EC0EF025C500F126C558
:1036F00001F127C502F128C503F10101100E046F85
:10370000000E056F000E066F000E076FD0EC30F054
:103710003DEC31F02AC182F40401300E8227A2EC84
:103720000EF02BC182F40401300E8227A2EC0EF0C1
:103730002CC182F40401300E8227A2EC0EF02DC1C0
:1037400082F40401300E8227A2EC0EF02EC182F426
:103750000401300E8227A2EC0EF02FC182F4040186
:10376000300E8227A2EC0EF030C182F40401300E3C
:103770008227A2EC0EF031C182F40401300E8227C0
:10378000A2EC0EF032C182F40401300E8227A2ECCA
:103790000EF033C182F40401300E8227A2EC0EF049
:1037A00007946EEF1EF0078404014C0E826FA2ECAA
:1037B0000EF00401320E826FA2EC0EF0D9EC36F05E
:1037C00007946EEF1EF0078438B0E9EF1BF0FCEFB2
:1037D0001BF0010E166E04014C0E826FA2EC0EF06F
:1037E0000401330E826FA2EC0EF036EC37F0000EBF
:1037F000166E079470EF1BF0020E166E36EC37F063
:103800008B800501010E306F3C0E316F01015E6B44
:103810005F6B606B616B626B636B646B656B666B3C
:10382000676B686B696B536B546BCF6ACE6A0F9A88
:103830000F9C0F9E030E166E04014C0E826FA2ECBD
:103840000EF00401330E826FA2EC0EF004012C0E78
:10385000826FA2EC0EF004012D0E826FA2EC0EF02E
:103860000401310E826FA2EC0EF0B5EF2AF036ECB7
:1038700037F0000E166E8B90B7EF2AF00784040124
:103880004C0E826FA2EC0EF00401340E826FA2EC9B
:103890000EF004012C0E826FA2EC0EF0F5EC31F06C
:1038A00084C32AF185C32BF186C32CF187C32DF184
:1038B00088C32EF189C32FF18AC330F18BC331F154
:1038C0008CC332F18DC333F10101296B02EC32F06C
:1038D00079EC31F0100E046F000E056F000E066FCC
:1038E000000E076FB0EC30F000C121F501C122F5E8
:1038F00002C123F503C124F5B8EC38F038C5AFF5A3
:1039000039C5B0F53AC5B1F53BC5B2F53CC5B3F51F
:103910003DC5B4F53EC5B5F5C7EC16F004012C0E57
:10392000826FA2EC0EF03FC500F140C501F141C528
:1039300002F142C503F10101000E046F000E056F94
:10394000010E066F000E076FD0EC30F03DEC31F049
:103950002967ADEF1CF0B2EF1CF004012D0E826F51
:10396000A2EC0EF030C182F40401300E8227A2ECEA
:103970000EF031C182F40401300E8227A2EC0EF069
:1039800004012E0E826FA2EC0EF032C182F404010B
:10399000300E8227A2EC0EF033C182F40401300E07
:1039A0008227A2EC0EF004012C0E826FA2EC0EF026
:1039B000B4EC31F043C500F144C501F1E1EC2BF06A
:1039C00004012C0E826FA2EC0EF0B4EC31F045C570
:1039D00000F13DEC31F031C182F40401300E822758
:1039E000A2EC0EF032C182F40401300E8227A2EC68
:1039F0000EF033C182F40401300E8227A2EC0EF0E7
:103A000004012C0E826FA2EC0EF037C5E8FFE8B877
:103A100006D00401300E826FA2EC0EF005D0040136
:103A2000310E826FA2EC0EF007946EEF1EF0F5ECF3
:103A300031F085C32AF186C32BF187C32CF188C3EB
:103A40002DF189C32EF18AC32FF18BC330F18CC3C2
:103A500031F18DC332F18EC333F10101296B02ECD8
:103A600032F079EC31F00101010E046F000E056FA8
:103A7000000E066F000E076F9FEC30F0100E046F03
:103A8000000E056F000E066F000E076FB0EC30F0F1
:103A900000C129F501C12AF502C12BF503C12CF59E
:103AA00060EC36F004014C0E826FA2EC0EF00401C3
:103AB000460E826FA2EC0EF004012C0E826FA2EC77
:103AC0000EF025C500F126C501F127C502F128C574
:103AD00003F10101100E046F000E056F000E066F5A
:103AE000000E076FD0EC30F03DEC31F02AC182F4CB
:103AF0000401300E8227A2EC0EF02BC182F40401E7
:103B0000300E8227A2EC0EF02CC182F40401300E9C
:103B10008227A2EC0EF02DC182F40401300E822720
:103B2000A2EC0EF02EC182F40401300E8227A2EC2A
:103B30000EF02FC182F40401300E8227A2EC0EF0A9
:103B400030C182F40401300E8227A2EC0EF031C1A4
:103B500082F40401300E8227A2EC0EF032C182F40E
:103B60000401300E8227A2EC0EF033C182F404016E
:103B7000300E8227A2EC0EF06EEF1EF038B0C3EFCD
:103B80001DF0020E166E36EC37F000011650020AD8
:103B9000D8B4E1EF1DF005012F51010AD8B4D7EFD9
:103BA0001DF015B2DCEF1DF081BADCEF1DF0000E48
:103BB000166E1584B7EF2AF0050E166E1584ADEF5C
:103BC00039F08B8001015E6B5F6B606B616B626BC8
:103BD000636B646B656B666B676B686B696B536B70
:103BE000546BCF6ACE6A0F9A0F9C0F9E030E166E0F
:103BF000B7EF2AF036EC37F005012F51010AD8B49F
:103C000008EF1EF015B20DEF1EF081BA0DEF1EF099
:103C1000000E166E1584B7EF2AF0050E166E158489
:103C2000ADEF39F004014C0E826FA2EC0EF00401EE
:103C3000350E826FA2EC0EF004012C0E826FA2EC06
:103C40000EF0B4EC31F00784B9C500F107943DECF7
:103C500031F031C182F40401300E8227A2EC0EF063
:103C600032C182F40401300E8227A2EC0EF033C17F
:103C700082F40401300E8227A2EC0EF06EEF1EF0EB
:103C8000F9EC36F0B4EC31F037C500F13DEC31F031
:103C900004014C0E826FA2EC0EF00401360E826F0E
:103CA000A2EC0EF004012C0E826FA2EC0EF031C1DA
:103CB00082F40401300E8227A2EC0EF032C182F4AD
:103CC0000401300E8227A2EC0EF033C182F404010D
:103CD000300E8227A2EC0EF06EEF1EF0ACEC0EF070
:103CE000B7EF2AF004014C0E826FA2EC0EF0040133
:103CF000500E826FA2EC0EF004012C0E826FA2EC2B
:103D00000EF085C32AF186C32BF187C32CF188C33B
:103D10002DF189C32EF18AC32FF18BC330F18CC3EF
:103D200031F18DC332F18EC333F1010102EC32F077
:103D300079EC31F003018451530A0DE00301845101
:103D40004D0A38E00401780E826FA2EC0EF0ACEC64
:103D50000EF0B7EF2AF00401530E826FA2EC0EF0C2
:103D6000250E0C6E00C10BF04DEC0BF0260E0C6E08
:103D700001C10BF04DEC0BF0270E0C6E02C10BF0E5
:103D80004DEC0BF0280E0C6E03C10BF04DEC0BF05C
:103D900000C157F501C158F502C159F503C15AF5E3
:103DA00000C15BF501C15CF502C15DF503C15EF5C3
:103DB0004FEF1FF004014D0E826FA2EC0EF0290EA2
:103DC0000C6E00C10BF04DEC0BF000C15FF500C1B3
:103DD00060F54FEF1FF004014C0E826FA2EC0EF065
:103DE0000401540E826FA2EC0EF004012C0E826FBF
:103DF000A2EC0EF084C32AF185C32BF186C32CF10B
:103E000087C32DF188C32EF189C32FF18AC330F106
:103E10008BC331F18DC332F18EC333F1010102EC5A
:103E200032F079EC31F00101000E046F000E056FE5
:103E3000010E066F000E076FB0EC30F0210E0C6E15
:103E400000C10BF04DEC0BF0220E0C6E01C10BF01B
:103E50004DEC0BF0230E0C6E02C10BF04DEC0BF091
:103E6000240E0C6E03C10BF04DEC0BF000C161F59C
:103E700001C162F502C163F503C164F54FEF1FF0A4
:103E800004014C0E826FA2EC0EF00401490E826F09
:103E9000A2EC0EF004012C0E826FA2EC0EF0250EA7
:103EA00064EC0BF0E8CF00F1260E64EC0BF0E8CFE9
:103EB00001F1270E64EC0BF0E8CF02F1280E64EC60
:103EC0000BF0E8CF03F13DEC31F000EC2FF00401F2
:103ED000730E826FA2EC0EF004012C0E826FA2EC26
:103EE0000EF0B4EC31F0290E64EC0BF0E8CF00F1E9
:103EF0003DEC31F000EC2FF004016D0E826FA2EC6E
:103F00000EF004012C0E826FA2EC0EF05BC500F1E6
:103F10005CC501F15DC502F15EC503F13DEC31F018
:103F200000EC2FF00401730E826FA2EC0EF004017E
:103F30002C0E826FA2EC0EF0B4EC31F060C500F1F3
:103F40003DEC31F000EC2FF004016D0E826FA2EC1D
:103F50000EF004012C0E826FA2EC0EF061C500F190
:103F600062C501F163C502F164C503F1D2EC2AF028
:103F700004012C0E826FA2EC0EF0ACEC0EF0B7EF49
:103F80002AF083C32AF184C32BF185C32CF186C3A5
:103F90002DF187C32EF188C32FF189C330F18AC375
:103FA00031F18BC332F18CC333F1010102EC32F0F9
:103FB00079EC31F0160E0C6E00C10BF04DEC0BF0ED
:103FC000170E0C6E01C10BF04DEC0BF0180E0C6EC1
:103FD00002C10BF04DEC0BF0190E0C6E03C10BF08F
:103FE0004DEC0BF000C18EF101C18FF102C190F1D7
:103FF00003C191F100C192F101C193F102C194F1A9
:1040000003C195F1A3EF20F083C32AF184C32BF100
:1040100085C32CF186C32DF187C32EF188C32FF100
:1040200089C330F18AC331F18BC332F18CC333F1D0
:10403000010102EC32F079EC31F000C18EF101C1E6
:104040008FF102C190F103C191F100C192F101C160
:1040500093F102C194F103C195F1A3EF20F083C362
:104060002AF184C32BF185C32CF186C32DF187C3BC
:104070002EF188C32FF189C330F18AC331F18CC38B
:1040800032F18DC333F1010102EC32F079EC31F001
:104090000101000E046F000E056F010E066F000E89
:1040A000076FB0EC30F01A0E0C6E00C10BF04DEC47
:1040B0000BF01B0E0C6E01C10BF04DEC0BF01C0E47
:1040C0000C6E02C10BF04DEC0BF01D0E0C6E03C11B
:1040D0000BF04DEC0BF000C196F101C197F102C15C
:1040E00098F103C199F1A3EF20F083C32AF184C3AF
:1040F0002BF185C32CF186C32DF187C32EF188C324
:104100002FF189C330F18AC331F18CC332F18DC3F1
:1041100033F1010102EC32F079EC31F00101000ED3
:10412000046F000E056F010E066F000E076FB0ECF6
:1041300030F000C196F101C197F102C198F103C1BD
:1041400099F1A3EF20F0160E64EC0BF0E8CF00F12C
:10415000170E64EC0BF0E8CF01F1180E64EC0BF0D5
:10416000E8CF02F1190E64EC0BF0E8CF03F13DEC5F
:1041700031F000EC2FF00401730E826FA2EC0EF010
:1041800004012C0E826FA2EC0EF08EC100F18FC1E3
:1041900001F190C102F191C103F13DEC31F000EC6D
:1041A0002FF00401730E826FA2EC0EF004012C0EAE
:1041B000826FA2EC0EF01A0E64EC0BF0E8CF00F167
:1041C0001B0E64EC0BF0E8CF01F11C0E64EC0BF05D
:1041D000E8CF02F11D0E64EC0BF0E8CF03F1D2EC56
:1041E0002AF004012C0E826FA2EC0EF096C100F1B1
:1041F00097C101F198C102F199C103F1D2EC2AF003
:10420000ACEC0EF0B7EF2AF00401690E826FA2EC5D
:104210000EF004012C0E826FA2EC0EF00101040ED0
:10422000006F000E016F000E026F000E036F3DEC79
:1042300031F02CC182F40401300E8227A2EC0EF082
:104240002DC182F40401300E8227A2EC0EF02EC1A3
:1042500082F40401300E8227A2EC0EF02FC182F40A
:104260000401300E8227A2EC0EF030C182F404016A
:10427000300E8227A2EC0EF031C182F40401300E20
:104280008227A2EC0EF032C182F40401300E8227A4
:10429000A2EC0EF033C182F40401300E8227A2ECAE
:1042A0000EF004012C0E826FA2EC0EF00101060E3E
:1042B000006F000E016F000E026F000E036F3DECE9
:1042C00031F02CC182F40401300E8227A2EC0EF0F2
:1042D0002DC182F40401300E8227A2EC0EF02EC113
:1042E00082F40401300E8227A2EC0EF02FC182F47A
:1042F0000401300E8227A2EC0EF030C182F40401DA
:10430000300E8227A2EC0EF031C182F40401300E8F
:104310008227A2EC0EF032C182F40401300E822713
:10432000A2EC0EF033C182F40401300E8227A2EC1D
:104330000EF004012C0E826FA2EC0EF00101510E62
:10434000006F000E016F000E026F000E036F3DEC58
:1043500031F02CC182F40401300E8227A2EC0EF061
:104360002DC182F40401300E8227A2EC0EF02EC182
:1043700082F40401300E8227A2EC0EF02FC182F4E9
:104380000401300E8227A2EC0EF030C182F4040149
:10439000300E8227A2EC0EF031C182F40401300EFF
:1043A0008227A2EC0EF032C182F40401300E822783
:1043B000A2EC0EF033C182F40401300E8227A2EC8D
:1043C0000EF004012C0E826FA2EC0EF0200EF86E9F
:1043D000F76AF66A04010900F5CF82F4A2EC0EF048
:1043E0000900F5CF82F4A2EC0EF00900F5CF82F4BB
:1043F000A2EC0EF00900F5CF82F4A2EC0EF0090059
:10440000F5CF82F4A2EC0EF00900F5CF82F4A2EC15
:104410000EF00900F5CF82F4A2EC0EF00900F5CF02
:1044200082F4A2EC0EF0ACEC0EF0B7EF2AF0835160
:10443000630AD8A4B5EF2AF08451610AD8A4B5EF75
:104440002AF085516C0AD8A4B5EF2AF08651410AAA
:104450003FE08651440A1BE08651420AD8B47BEF04
:1044600022F08651350AD8B441EF2CF08651360A35
:10447000D8B496EF2CF08651370AD8B4FFEF2CF061
:104480008651380AD8B45DEF2DF0B5EF2AF00798C1
:10449000079A04017A0E826FA2EC0EF00401780EE6
:1044A000826FA2EC0EF00401640E826FA2EC0EF09B
:1044B0000401550E826FA2EC0EF064EF22F00401AD
:1044C0004C0E826FA2EC0EF0ACEC0EF0B7EF2AF0BF
:1044D0000788079A04017A0E826FA2EC0EF004019D
:1044E000410E826FA2EC0EF00401610E826FA2EC0D
:1044F0000EF058EF22F00798078A04017A0E826FB7
:10450000A2EC0EF00401420E826FA2EC0EF0040148
:10451000610E826FA2EC0EF058EF22F00101666787
:1045200099EF22F0676799EF22F0686799EF22F020
:10453000696716D001014F67A5EF22F05067A5EF1C
:1045400022F05167A5EF22F052670AD00101000E58
:10455000006F000E016F000E026F000E036F12005D
:1045600011B80AD00101620E046F010E056F000E32
:10457000066F000E076F09D00101A70E046F020E2F
:10458000056F000E066F000E076F66C100F167C170
:1045900001F168C102F169C103F19FEC30F003BF82
:1045A00042EF23F0119A119C0101000E046FA80E36
:1045B000056F550E066F020E076F66C100F167C1E9
:1045C00001F168C102F169C103F166C18AF167C1F5
:1045D0008BF168C18CF169C18DF19FEC30F003BFA4
:1045E0000BD00101000E8A6FA80E8B6F550E8C6FD9
:1045F000020E8D6F118A119C0E0E64EC0BF0E8CF49
:1046000018F10F0E64EC0BF0E8CF19F1100E64EC0A
:104610000BF0E8CF1AF1110E64EC0BF0E8CF1BF1B0
:10462000E8EC2FF08AC104F18BC105F18CC106F1D1
:104630008DC107F19FEC30F00782ACEC2FF0E8EC75
:104640002FF00792ACEC2FF08AC100F18BC101F181
:104650008CC102F18DC103F10792ACEC2FF0CC0EAE
:10466000046FE00E056F870E066F050E076F9FEC57
:1046700030F000C118F101C119F102C11AF103C1F2
:104680001BF140D013AA47EF23F0138E139A119C0D
:10469000119A0101800E006F1A0E016F060E026F53
:1046A000000E036F4FC104F150C105F151C106F175
:1046B00052C107F19FEC30F003AF05D0B4EC31F0FC
:1046C000118C119A12000E0E64EC0BF0E8CF18F169
:1046D0000F0E64EC0BF0E8CF19F1100E64EC0BF048
:1046E000E8CF1AF1110E64EC0BF0E8CF1BF14FC1CB
:1046F00000F150C101F151C102F152C103F1078231
:10470000ACEC2FF018C100F119C101F11AC102F18E
:104710001BC103F112000784BAC166F1BBC167F186
:10472000BCC168F1BDC169F14BC14FF14CC150F141
:104730004DC151F14EC152F157C159F158C15AF111
:10474000079401016667ACEF23F06767ACEF23F0D5
:104750006867ACEF23F0696716D001014F67B8EFC7
:1047600023F05067B8EF23F05167B8EF23F052679A
:104770000AD00101000E006F000E016F000E026FE3
:10478000000E036F120011B80AD00101620E046F0F
:10479000010E056F000E066F000E076F09D00101B4
:1047A000A70E046F020E056F000E066F000E076F56
:1047B00066C100F167C101F168C102F169C103F18D
:1047C0009FEC30F003BF44EF24F00101000E046FB2
:1047D000A80E056F550E066F020E076F66C100F139
:1047E00067C101F168C102F169C103F166C18AF1D3
:1047F00067C18BF168C18CF169C18DF19FEC30F01C
:1048000003BF09D00101000E8A6FA80E8B6F550EF1
:104810008C6F020E8D6FE8EC2FF000C104F101C126
:1048200005F102C106F103C107F1000E006FA00EF1
:10483000016F980E026F7B0E036FD0EC30F000C159
:1048400018F101C119F102C11AF103C11BF1000EE7
:10485000006FA00E016F980E026F7B0E036F8AC16E
:1048600004F18BC105F18CC106F18DC107F1D0ECCB
:1048700030F018C104F119C105F11AC106F11BC1CC
:1048800007F19FEC30F012000101A80E006F610EDD
:10489000016F000E026F000E036F4FC104F150C193
:1048A00005F151C106F152C107F19FEC30F003AFA1
:1048B0000AD00101A80E006F610E016F000E026F99
:1048C000000E036F00D0C80E006FAF0E016F000E18
:1048D000026F000E036F4FC104F150C105F151C1C9
:1048E00006F152C107F1B0EC30F012000784BAC1F2
:1048F00066F1BBC167F1BCC168F1BDC169F14BC1D3
:104900004FF14CC150F14DC151F14EC152F157C15F
:1049100059F158C15AF107940101666797EF24F0E5
:10492000676797EF24F0686797EF24F0696716D000
:1049300001014F67A3EF24F05067A3EF24F0516704
:10494000A3EF24F052670AD00101000E006F000EA1
:10495000016F000E026F000E036F120011B80AD033
:104960000101620E046F010E056F000E066F000E4E
:10497000076F09D00101A70E046F020E056F000E2C
:10498000066F000E076F66C100F167C101F168C1D3
:1049900002F169C103F19FEC30F003BF59EF25F03C
:1049A0000101000E046FA80E056F550E066F020E72
:1049B000076F66C100F167C101F168C102F169C109
:1049C00003F166C18AF167C18BF168C18CF169C1DD
:1049D0008DF19FEC30F003BF09D00101000E8A6F0A
:1049E000A80E8B6F550E8C6F020E8D6F010E006F2F
:1049F000000E016F000E026F000E036F8AC104F1FA
:104A00008BC105F18CC106F18DC107F1D0EC30F0FE
:104A100018C104F119C105F11AC106F11BC107F152
:104A20003DEC31F02AC182F40401300E8227A2EC61
:104A30000EF02BC182F40401300E8227A2EC0EF09E
:104A40002CC182F40401300E8227A2EC0EF02DC19D
:104A500082F40401300E8227A2EC0EF02EC182F403
:104A60000401300E8227A2EC0EF02FC182F4040163
:104A7000300E8227A2EC0EF030C182F40401300E19
:104A80008227A2EC0EF031C182F40401300E82279D
:104A9000A2EC0EF032C182F40401300E8227A2ECA7
:104AA0000EF033C182F40401300E8227A2EC0EF026
:104AB00012004FC100F150C101F151C102F152C1C8
:104AC00003F101013DEC31F000EC2FF01200040184
:104AD000730E826FA2EC0EF004012C0E826FA2EC1A
:104AE0000EF0078462C166F163C167F164C168F1C9
:104AF00065C169F14BC14FF14CC150F14DC151F14C
:104B00004EC152F157C159F158C15AF107948DEC79
:104B100025F0ACEC0EF0B7EF2AF066C100F167C1EA
:104B200001F168C102F169C103F101013DEC31F00D
:104B300000EC2FF00401630E826FA2EC0EF0040172
:104B40002C0E826FA2EC0EF04FC100F150C101F1AA
:104B500051C102F152C103F101013DEC31F000EC11
:104B60002FF00401660E826FA2EC0EF004012C0EF1
:104B7000826FA2EC0EF0B4EC31F059C100F15AC1D1
:104B800001F101013DEC31F000EC2FF00401740E55
:104B9000826FA2EC0EF0120010820401530E826F9D
:104BA000A2EC0EF004012C0E826FA2EC0EF083C377
:104BB0002AF184C32BF185C32CF186C32DF187C361
:104BC0002EF188C32FF189C330F18AC331F18BC331
:104BD00032F18CC333F1010102EC32F079EC31F0A7
:104BE00000C166F101C167F102C168F103C169F159
:104BF0008EC32AF18FC32BF190C32CF191C32DF1F9
:104C000092C32EF193C32FF194C330F195C331F1C8
:104C100096C332F197C333F1010102EC32F079EC23
:104C200031F000C14FF101C150F102C151F103C196
:104C300052F1F5EC31F099C32FF19AC330F19BC3D7
:104C400031F19CC332F19DC333F1010102EC32F02A
:104C500079EC31F000C159F101C15AF18DEC25F028
:104C600004012C0E826FA2EC0EF047EF26F0118E9D
:104C70001CA002D01CAE108C1BBE02D01BA4108E38
:104C800003018251520A02E10F8201D00F92825138
:104C9000750A02E1108401D010948251550A02E194
:104CA000108601D010968351310A03E113821384D8
:104CB00002D01392139403018351660A01E056D087
:104CC0000401660E826FA2EC0EF004012C0E826FBE
:104CD000A2EC0EF08BEC23F03DEC31F02AC182F413
:104CE0000401300E8227A2EC0EF02BC182F40401E5
:104CF000300E8227A2EC0EF02CC182F40401300E9B
:104D00008227A2EC0EF02DC182F40401300E82271E
:104D1000A2EC0EF02EC182F40401300E8227A2EC28
:104D20000EF02FC182F40401300E8227A2EC0EF0A7
:104D300030C182F40401300E8227A2EC0EF031C1A2
:104D400082F40401300E8227A2EC0EF032C182F40C
:104D50000401300E8227A2EC0EF033C182F404016C
:104D6000300E8227A2EC0EF0B5EF2AF011A003D08E
:104D700011A401D01084078410B220EF27F010A4F2
:104D800004EF27F0BAC166F1BBC167F1BCC168F19D
:104D9000BDC169F1BEC16AF1BFC16BF1C0C16CF1A7
:104DA000C1C16DF1C2C16EF1C3C16FF1C4C170F177
:104DB000C5C171F1C6C172F1C7C173F1C8C174F147
:104DC000C9C175F1CAC176F1CBC177F1CCC178F117
:104DD000CDC179F1CEC17AF1CFC17BF1D0C17CF1E7
:104DE000D1C17DF1D2C17EF1D3C17FF1D4C180F1B7
:104DF000D5C181F1D6C182F1D7C183F1D8C184F187
:104E0000D9C185F10CEF27F062C166F163C167F18A
:104E100064C168F165C169F1BAC186F1BBC187F1AE
:104E2000BCC188F1BDC189F14BC14FF14CC150F1FA
:104E30004DC151F14EC152F157C159F158C15AF10A
:104E400007940FA042EF27F0010196672FEF27F09C
:104E500097672FEF27F098672FEF27F0996733EFC9
:104E600027F042EF27F08EEC22F096C104F197C1B3
:104E700005F198C106F199C107F19FEC30F003BF2D
:104E80007BEF2AF08EEC22F00101000E046F000E81
:104E9000056F010E066F000E076FD0EC30F011A009
:104EA0002AD011A228D03DEC31F0296701D005D0DD
:104EB00004012D0E826FA2EC0EF030C182F40401C9
:104EC000300E8227A2EC0EF031C182F40401300EC4
:104ED0008227A2EC0EF032C182F40401300E822748
:104EE000A2EC0EF033C182F40401300E8227A2EC52
:104EF0000EF0ACEC0EF012A8C5D012981DC01EF03A
:104F00001E3A1E42070E1E1600011E50000AD8B49B
:104F10000EEF28F000011E50010AD8B49AEF27F0D6
:104F200000011E50020AD8B498EF27F040EF28F095
:104F300040EF28F0B4EC31F02EC001F12FC000F1A9
:104F4000D89001330033D890013300330101630E50
:104F5000046F000E056F000E066F000E076FD0EC99
:104F600030F0280E046F000E056F000E066F000E65
:104F7000076F9FEC30F000C131F0B4EC31F02CC081
:104F800001F1019F019D2DC000F10101A40E046FEC
:104F9000000E056F000E066F000E076FD0EC30F0AC
:104FA00000C130F000C104F101C105F102C106F1F8
:104FB00003C107F1640E006F000E016F000E026F57
:104FC000000E036F9FEC30F0050E046F000E056FAE
:104FD000000E066F000E076FD0EC30F000C104F138
:104FE00001C105F102C106F103C107F1B4EC31F0D2
:104FF00031C000F19FEC30F000C132F032C0E8FF68
:10500000050F315C03E78A8440EF28F032C0E8FFE7
:105010000A0F315C01E68A9440EF28F000C124F1C8
:1050200001C125F102C126F103C127F1B4EC31F031
:10503000BAEC31F01D501F0BE8CF00F10101640EF6
:10504000046F000E056F000E066F000E076FB0ECC8
:1050500030F024C104F125C105F126C106F127C1B4
:1050600007F19FEC30F003BF02D08A9401D08A840C
:1050700024C100F125C101F126C102F127C103F1CC
:10508000B7EF2AF000C124F101C125F102C126F1D8
:1050900003C127F110AE4DD0109E00C108F101C12F
:1050A00009F102C10AF103C10BF13DEC31F030C14D
:1050B000E2F131C1E3F132C1E4F133C1E5F108C1FC
:1050C00000F109C101F10AC102F10BC103F10101B3
:1050D0006C0E046F070E056F000E066F000E076F53
:1050E0009FEC30F003BF04D00101550EE66F1CD0D9
:1050F00008C100F109C101F10AC102F10BC103F1BC
:105100000101A40E046F060E056F000E066F000E5F
:10511000076F9FEC30F003BF04D001017F0EE66FF4
:1051200003D00101FF0EE66F1F8E11AE7BEF2AF058
:10513000119E24C100F125C101F126C102F127C150
:1051400003F111A005D011A203D00FB07BEF2AF01C
:1051500010A4B2EF28F00401750E826FA2EC0EF0DD
:10516000B7EF28F00401720E826FA2EC0EF004017A
:105170002C0E826FA2EC0EF03DEC31F02967C6EFE9
:1051800028F00401200E826FC9EF28F004012D0ED3
:10519000826FA2EC0EF030C182F40401300E82273F
:1051A000A2EC0EF031C182F40401300E8227A2EC91
:1051B0000EF004012E0E826FA2EC0EF032C182F4CA
:1051C0000401300E8227A2EC0EF033C182F40401F8
:1051D000300E8227A2EC0EF004016D0E826FA2EC5D
:1051E0000EF004012C0E826FA2EC0EF04FC100F104
:1051F00050C101F151C102F152C103F101013DEC75
:1052000031F000EC2FF00401480E826FA2EC0EF09A
:1052100004017A0E826FA2EC0EF004012C0E826F54
:10522000A2EC0EF066C100F167C101F168C102F1A4
:1052300069C103F101013DEC31F000EC2FF00401F4
:10524000630E826FA2EC0EF004012C0E826FA2ECB2
:105250000EF066C100F167C101F168C102F169C1D8
:1052600003F101010A0E046F000E056F000E066FB8
:10527000000E076FB0EC30F0000E046F120E056FD9
:10528000000E066F000E076FD0EC30F03DEC31F0F1
:105290002AC182F40401300E8227A2EC0EF02BC149
:1052A00082F40401300E8227A2EC0EF02CC182F4AD
:1052B0000401300E8227A2EC0EF02DC182F404010D
:1052C000300E8227A2EC0EF02EC182F40401300EC3
:1052D0008227A2EC0EF02FC182F40401300E822747
:1052E000A2EC0EF030C182F40401300E8227A2EC51
:1052F0000EF004012E0E826FA2EC0EF031C182F48A
:105300000401300E8227A2EC0EF032C182F40401B7
:10531000300E8227A2EC0EF033C182F40401300E6D
:105320008227A2EC0EF00401730E826FA2EC0EF045
:1053300004012C0E826FA2EC0EF0B4EC31F059C1D6
:1053400000F15AC101F1E1EC2BF013A2F7EF29F0C3
:1053500004012C0E826FA2EC0EF086C166F187C1AB
:1053600067F188C168F189C169F18EEC22F0010111
:10537000000E046F000E056F010E066F000E076F22
:10538000D0EC30F03DEC31F02967CCEF29F004018E
:10539000200E826FCFEF29F004012D0E826FA2EC58
:1053A0000EF030C182F40401300E8227A2EC0EF020
:1053B00031C182F40401300E8227A2EC0EF0040108
:1053C0002E0E826FA2EC0EF032C182F40401300E78
:1053D0008227A2EC0EF033C182F40401300E822742
:1053E000A2EC0EF004016D0E826FA2EC0EF0030130
:1053F0008351460A01E007D004012C0E826FA2EC13
:105400000EF076EC24F013A42AEF2AF004012C0EFF
:10541000826FA2EC0EF013AC18EF2AF00401500ECC
:10542000826FA2EC0EF0139C1398139A2AEF2AF0C5
:1054300013AE25EF2AF00401460E826FA2EC0EF0A7
:10544000139E1398139A2AEF2AF00401530E826FC9
:10545000A2EC0EF038B041EF2AF004012C0E826F5E
:10546000A2EC0EF08BB03CEF2AF00401440E826FE8
:10547000A2EC0EF041EF2AF00401530E826FA2EC71
:105480000EF00FB247EF2AF00FA079EF2AF00401D7
:105490002C0E826FA2EC0EF0200EF86EF76AF66A00
:1054A00004010900F5CF82F4A2EC0EF00900F5CF5B
:1054B00082F4A2EC0EF00900F5CF82F4A2EC0EF01B
:1054C0000900F5CF82F4A2EC0EF00900F5CF82F4CA
:1054D000A2EC0EF00900F5CF82F4A2EC0EF0090068
:1054E000F5CF82F4A2EC0EF00900F5CF82F4A2EC25
:1054F0000EF0ACEC0EF00F90109E1298B7EF2AF061
:105500000401630E826FA2EC0EF004012C0E826F78
:10551000A2EC0EF0BDEC2AF004012C0E826FA2EC7E
:105520000EF030EC2BF004012C0E826FA2EC0EF08A
:10553000ACEC2BF004012C0E826FA2EC0EF00101FA
:10554000F80E006FCD0E016F660E026F030E036F33
:10555000D2EC2AF004012C0E826FA2EC0EF0C2EC09
:105560002BF0ACEC0EF0B7EF2AF0ACEC0EF0030130
:10557000C26B07901092C6EF2DF0D8900E0E64EC1F
:105580000BF0E8CF00F10F0E64EC0BF0E8CF01F167
:10559000100E64EC0BF0E8CF02F1110E64EC0BF08E
:1055A000E8CF03F10101000E046F000E056F010E3C
:1055B000066F000E076FD0EC30F03DEC31F02AC1E1
:1055C00082F40401300E8227A2EC0EF02BC182F48B
:1055D0000401300E8227A2EC0EF02CC182F40401EB
:1055E000300E8227A2EC0EF02DC182F40401300EA1
:1055F0008227A2EC0EF02EC182F40401300E822725
:10560000A2EC0EF02FC182F40401300E8227A2EC2E
:105610000EF030C182F40401300E8227A2EC0EF0AD
:1056200031C182F40401300E8227A2EC0EF0040195
:105630002E0E826FA2EC0EF032C182F40401300E05
:105640008227A2EC0EF033C182F40401300E8227CF
:10565000A2EC0EF004016D0E826FA2EC0EF01200AF
:10566000120E64EC0BF0E8CF00F1130E64EC0BF0BB
:10567000E8CF01F1140E64EC0BF0E8CF02F1150E47
:1056800064EC0BF0E8CF03F101010A0E046F000E89
:10569000056F000E066F000E076FB0EC30F0000EC5
:1056A000046F120E056F000E066F000E076FD0EC30
:1056B00030F03DEC31F02AC182F40401300E822733
:1056C000A2EC0EF02BC182F40401300E8227A2EC72
:1056D0000EF02CC182F40401300E8227A2EC0EF0F1
:1056E0002DC182F40401300E8227A2EC0EF02EC1EF
:1056F00082F40401300E8227A2EC0EF02FC182F456
:105700000401300E8227A2EC0EF030C182F40401B5
:10571000300E8227A2EC0EF004012E0E826FA2EC56
:105720000EF031C182F40401300E8227A2EC0EF09B
:1057300032C182F40401300E8227A2EC0EF033C194
:1057400082F40401300E8227A2EC0EF00401730EE5
:10575000826FA2EC0EF012000A0E64EC0BF0E8CFA0
:1057600000F10B0E64EC0BF0E8CF01F10C0E64ECD1
:105770000BF0E8CF02F10D0E64EC0BF0E8CF03F173
:10578000E1EF2BF0060E64EC0BF0E8CF00F1070E12
:1057900064EC0BF0E8CF01F1080E64EC0BF0E8CFFD
:1057A00002F1090E64EC0BF0E8CF03F1E1EF2BF00E
:1057B0000101B4EC31F0078457C100F158C101F187
:1057C00007940101E80E046F800E056F000E066F4E
:1057D000000E076FB0EC30F0000E046F040E056F82
:1057E000000E066F000E076FD0EC30F0880E046FCD
:1057F000130E056F000E066F000E076F9FEC30F062
:105800000A0E046F000E056F000E066F000E076F84
:10581000D0EC30F03DEC31F00101296715EF2CF0B0
:105820000401200E826F18EF2CF004012D0E826F00
:10583000A2EC0EF030C182F40401300E8227A2ECFB
:105840000EF031C182F40401300E8227A2EC0EF07A
:1058500032C182F40401300E8227A2EC0EF0040162
:105860002E0E826FA2EC0EF033C182F40401300ED2
:105870008227A2EC0EF00401430E826FA2EC0EF020
:10588000120087C32AF188C32BF189C32CF18AC384
:105890002DF18BC32EF18CC32FF18DC330F18EC34C
:1058A00031F190C332F191C333F10101296B02EC64
:1058B00032F079EC31F00101000E046F000E056F3B
:1058C000010E066F000E076FB0EC30F00E0E0C6E7E
:1058D00000C10BF04DEC0BF00F0E0C6E01C10BF084
:1058E0004DEC0BF0100E0C6E02C10BF04DEC0BF0FA
:1058F000110E0C6E03C10BF04DEC0BF004017A0E8F
:10590000826FA2EC0EF004012C0E826FA2EC0EF05E
:105910000401350E826FA2EC0EF004012C0E826F92
:10592000A2EC0EF0BDEC2AF064EF22F087C32AF15E
:1059300088C32BF189C32CF18AC32DF18BC32EF1BF
:105940008CC32FF18DC330F18EC331F190C332F18E
:1059500091C333F10101296B02EC32F079EC31F0A3
:10596000880E046F130E056F000E066F000E076F92
:10597000A4EC30F0000E046F040E056F000E066FED
:10598000000E076FB0EC30F00101E80E046F800EDE
:10599000056F000E066F000E076FD0EC30F00A0E98
:1059A0000C6E00C10BF04DEC0BF00B0E0C6E01C138
:1059B0000BF04DEC0BF00C0E0C6E02C10BF04DEC2D
:1059C0000BF00D0E0C6E03C10BF04DEC0BF004014F
:1059D0007A0E826FA2EC0EF004012C0E826FA2EC04
:1059E0000EF00401360E826FA2EC0EF004012C0EB4
:1059F000826FA2EC0EF0ACEC2BF064EF22F087C3C8
:105A00002AF188C32BF189C32CF18AC32DF18BC3F2
:105A10002EF18CC32FF18DC330F18FC331F190C3C0
:105A200032F191C333F1010102EC32F079EC31F043
:105A3000000E046F120E056F000E066F000E076F4A
:105A4000B0EC30F001010A0E046F000E056F000E7D
:105A5000066F000E076FD0EC30F0120E0C6E00C116
:105A60000BF04DEC0BF0130E0C6E01C10BF04DEC76
:105A70000BF0140E0C6E02C10BF04DEC0BF0150E7A
:105A80000C6E03C10BF04DEC0BF004017A0E826F2B
:105A9000A2EC0EF004012C0E826FA2EC0EF00401B9
:105AA000370E826FA2EC0EF004012C0E826FA2EC76
:105AB0000EF030EC2BF064EF22F087C32AF188C39C
:105AC0002BF189C32CF18AC32DF18BC32EF18CC32A
:105AD0002FF18DC330F18EC331F190C332F191C3F8
:105AE00033F10101296B02EC32F079EC31F0880ED0
:105AF000046F130E056F000E066F000E076FA4EC07
:105B000030F0000E046F040E056F000E066F000EDD
:105B1000076FB0EC30F00101E80E046F800E056FE6
:105B2000000E066F000E076FD0EC30F0060E0C6E04
:105B300000C10BF04DEC0BF0070E0C6E01C10BF029
:105B40004DEC0BF0080E0C6E02C10BF04DEC0BF09F
:105B5000090E0C6E03C10BF04DEC0BF004017A0E34
:105B6000826FA2EC0EF004012C0E826FA2EC0EF0FC
:105B70000401380E826FA2EC0EF004012C0E826F2D
:105B8000A2EC0EF0C2EC2BF064EF22F007A839EF84
:105B90002EF00101800E006F1A0E016F060E026FCB
:105BA000000E036F4BC104F14CC105F14DC106F16C
:105BB0004EC107F19FEC30F003BF7FEF2EF0FAECFF
:105BC0002EF04BC100F14CC101F14DC102F14EC1AB
:105BD00003F10782ACEC2FF018C104F119C105F1F3
:105BE0001AC106F11BC107F1F80E006FCD0E016F4F
:105BF000660E026F030E036F9FEC30F00E0E0C6EFC
:105C000000C10BF04DEC0BF00F0E0C6E01C10BF050
:105C10004DEC0BF0100E0C6E02C10BF04DEC0BF0C6
:105C2000110E0C6E03C10BF04DEC0BF0078401015B
:105C3000B4EC31F057C100F158C101F107940A0EDC
:105C40000C6E00C10BF04DEC0BF00B0E0C6E01C195
:105C50000BF04DEC0BF00C0E0C6E02C10BF04DEC8A
:105C60000BF00D0E0C6E03C10BF04DEC0BF07FEF43
:105C70002EF007AA7FEF2EF007840101B4EC31F07B
:105C800057C100F158C101F10794060E0C6E00C116
:105C90000BF04DEC0BF0070E0C6E01C10BF04DEC50
:105CA0000BF0080E0C6E02C10BF04DEC0BF0090E60
:105CB0000C6E03C10BF04DEC0BF0078462C100F1D8
:105CC00063C101F164C102F165C103F10794120ED1
:105CD0000C6E00C10BF04DEC0BF0130E0C6E01C1FD
:105CE0000BF04DEC0BF0140E0C6E02C10BF04DECF2
:105CF0000BF0150E0C6E03C10BF04DEC0BF007987A
:105D0000079A0401805181197F0B0DE09EA8FED7F0
:105D100014EE00F081517F0BE126E750812B0F013B
:105D2000AD6E81EF2EF005012F51000AD8B4C2EFFD
:105D30002EF081BAA7EF2EF015B2C2EF2EF00501BA
:105D40002F51010AD8B4C0EF2EF0B9EF2EF00501A3
:105D50002F51000AD8B4ADEF39F005012F51010AD7
:105D6000D8B4C0EF2EF000011650050AD8B4ADEF3C
:105D700039F081B8C2EF2EF02FEC33F0D5EC33F0D0
:105D800044EC39F0D0EF0DF018C100F119C101F168
:105D90001AC102F11BC103F1000E046F000E056F62
:105DA000010E066F000E076FD0EC30F029A1EFEF67
:105DB0002EF02051D8B4EFEF2EF018C100F119C128
:105DC00001F11AC102F11BC103F1000E046F000EB4
:105DD000056F0A0E066F000E076FD0EC30F0120050
:105DE000010104510013055101130651021307511B
:105DF000031312000101186B196B1A6B1B6B120055
:105E00002AC182F40401300E8227A2EC0EF02BC1CD
:105E100082F40401300E8227A2EC0EF02CC182F431
:105E20000401300E8227A2EC0EF02DC182F4040191
:105E3000300E8227A2EC0EF02EC182F40401300E47
:105E40008227A2EC0EF02FC182F40401300E8227CB
:105E5000A2EC0EF030C182F40401300E8227A2ECD5
:105E60000EF031C182F40401300E8227A2EC0EF054
:105E700032C182F40401300E8227A2EC0EF033C14D
:105E800082F40401300E8227A2EC0EF012002FC122
:105E900082F40401300E8227A2EC0EF030C182F4AD
:105EA0000401300E8227A2EC0EF031C182F404010D
:105EB000300E8227A2EC0EF032C182F40401300EC3
:105EC0008227A2EC0EF033C182F40401300E822747
:105ED000A2EC0EF01200060E216E060E226E060EC9
:105EE000236E212E71EF2FF0222E71EF2FF0232E33
:105EF00071EF2FF08B84020E216E020E226E020EC5
:105F0000236E212E81EF2FF0222E81EF2FF0232EF2
:105F100081EF2FF08B941200FF0E226E22C023F02F
:105F2000030E216E8B84212E92EF2FF0030E216E33
:105F3000232E92EF2FF08B9422C023F0030E216EBC
:105F4000212EA0EF2FF0030E216E233EA0EF2FF0A5
:105F5000222E8EEF2FF012000101005305E10153B4
:105F600003E1025301E1002B6FEC30F0B4EC31F0AF
:105F70003951006F3A51016F420E046F4B0E056F9D
:105F8000000E066F000E076FB0EC30F000C104F198
:105F900001C105F102C106F103C107F118C100F109
:105FA00019C101F11AC102F11BC103F107B2DDEF02
:105FB0002FF0A4EC30F0DFEF2FF09FEC30F000C1B9
:105FC00018F101C119F102C11AF103C11BF112004C
:105FD000B4EC31F059C100F15AC101F1060E64EC84
:105FE0000BF0E8CF04F1070E64EC0BF0E8CF05F1FD
:105FF000080E64EC0BF0E8CF06F1090E64EC0BF030
:10600000E8CF07F19FEC30F000C124F101C125F188
:1060100002C126F103C127F1290E046F000E056F9E
:10602000000E066F000E076FB0EC30F0EE0E046F3E
:10603000430E056F000E066F000E076FA4EC30F0E4
:1060400024C104F125C105F126C106F127C107F1DC
:10605000B0EC30F000C11CF101C11DF102C11EF114
:1060600003C11FF1120E64EC0BF0E8CF04F1130E24
:1060700064EC0BF0E8CF05F1140E64EC0BF0E8CF04
:1060800006F1150E64EC0BF0E8CF07F10D0E006F72
:10609000000E016F000E026F000E036FB0EC30F0C7
:1060A000180E046F000E056F000E066F000E076FCE
:1060B000D0EC30F01CC104F11DC105F11EC106F188
:1060C0001FC107F1A4EC30F06A0E046F2A0E056FB1
:1060D000000E066F000E076F9FEC30F01200BF0E2F
:1060E000FA6E200E3A6F396BD890003701370237BD
:1060F0000337D8B080EF30F03A2F75EF30F0390722
:106100003A070353D8B412000331070B80093F6FDD
:1061100003390F0B010F396F80EC5FF0406F3905C9
:1061200080EC5FF0405D405F396B3F33D8B039277A
:1061300039333FA995EF30F0405139271200010162
:10614000D9EC31F0D8B01200010103510719346FB6
:106150009CEC31F0D8900751031934AF800F120036
:106160000101346BC0EC31F0D8A0D6EC31F0D8B0DE
:106170001200ABEC31F0B4EC31F01F0E366FECECEA
:1061800031F00B35D8B09CEC31F0D8A00335D8B045
:106190001200362FBFEF30F034B1C3EC31F01200F3
:1061A0000101346B04510511061107110008D8A034
:1061B000C0EC31F0D8A0D6EC31F0D8B01200086BAA
:1061C000096B0A6B0B6BECEC31F01F0E366FECECCD
:1061D00031F007510B5DD8A4FAEF30F006510A5D9B
:1061E000D8A4FAEF30F00551095DD8A4FAEF30F0E9
:1061F0000451085DD8A00DEF31F00451085F05513E
:10620000D8A0053D095F0651D8A0063D0A5F075199
:10621000D8A0073D0B5FD8900081362FE7EF30F014
:1062200034B1C3EC31F0346BC0EC31F0D890F0EC09
:1062300031F007510B5DD8A42AEF31F006510A5D09
:10624000D8A42AEF31F00551095DD8A42AEF31F026
:106250000451085DD8A039EF31F0003F39EF31F03B
:10626000013F39EF31F0023F39EF31F0032BD8B461
:10627000120034B1C3EC31F012000101346BC0ECF8
:1062800031F0D8B01200F5EC31F0200E366F003747
:1062900001370237033711EE33F00A0E376FE73656
:1062A0000A0EE75CD8B0E76EE552372F4FEF31F0BA
:1062B000362F47EF31F034B12981D8901200F5EC38
:1062C00031F0200E366F003701370237033711EEF9
:1062D00033F00A0E376FE7360A0EE75CD8B0E76E88
:1062E000E552372F6BEF31F0362F63EF31F0D89056
:1062F000120001010A0E346F200E366F11EE29F0E4
:106300003451376F0A0ED890E652D8B0E726E732FC
:10631000372F84EF31F00333023301330033362F4C
:106320007EEF31F0E750FF0FD8A00335D8B0120050
:1063300029B1C3EC31F01200045100270551D8B047
:10634000053D01270651D8B0063D02270751D8B0B8
:10635000073D032712000051086F0151096F0251D8
:106360000A6F03510B6F12000101006B016B026B8E
:10637000036B12000101046B056B066B076B1200C7
:106380000335D8A012000351800B001F011F021F0C
:10639000031F003FD3EF31F0013FD3EF31F0023F55
:1063A000D3EF31F0032B342B032512000735D8A08F
:1063B00012000751800B041F051F061F071F043F13
:1063C000E9EF31F0053FE9EF31F0063FE9EF31F059
:1063D000072B342B0725120000370137023703370C
:1063E000083709370A370B3712000101296B2A6B6E
:1063F0002B6B2C6B2D6B2E6B2F6B306B316B326BD1
:10640000336B120001012A510F0B2A6F2B510F0B16
:106410002B6F2C510F0B2C6F2D510F0B2D6F2E51FD
:106420000F0B2E6F2F510F0B2F6F30510F0B306F43
:1064300031510F0B316F32510F0B326F33510F0B44
:10644000336F120000C124F101C125F102C126F110
:1064500003C127F104C100F105C101F106C102F138
:1064600007C103F124C104F125C105F126C106F1DC
:1064700027C107F1120000012550FE0AD8B449EFE8
:1064800032F000012550FD0AD8B449EF32F089847A
:1064900001D08994000EC76E220EC66E050EE82E3E
:1064A000FED7120000012550FE0AD8B460EF32F08A
:1064B00000012550FD0AD8B460EF32F0899401D074
:1064C0008984050EE82EFED712003BEC32F0000165
:1064D0002550FD0AD8B478EF32F09E96C69E000E85
:1064E000C96EFF0E9EB602D0E82EFCD781EF32F0C7
:1064F0009E96C69E010EC96EFF0E9EB602D0E82E75
:10650000FCD79E96C69E000EC96EFF0E9EB602D0A8
:10651000E82EFCD7C9CFAFF59E96C69E000EC96E79
:10652000FF0E9EB602D0E82EFCD7C9CFB0F59E96DE
:10653000C69E000EC96EFF0E9EB602D0E82EFCD796
:10654000C9CFB1F59E96C69E000EC96EFF0E9EB6CF
:1065500002D0E82EFCD7C9CFB2F59E96C69E000E9B
:10656000C96EFF0E9EB602D0E82EFCD7C9CFB3F598
:106570009E96C69E000EC96EFF0E9EB602D0E82EF5
:10658000FCD7C9CFB4F59E96C69E000EC96EFF0E0D
:106590009EB602D0E82EFCD7C9CFB5F552EC32F04A
:1065A00012003BEC32F000012550FD0AD8B4E4EFB4
:1065B00032F09E96C69E800EC96EFF0E9EB602D029
:1065C000E82EFCD7EDEF32F09E96C69E810EC96E86
:1065D000FF0E9EB602D0E82EFCD79E96C69EAFC593
:1065E000C9FFFF0E9EB602D0E82EFCD79E96C69E2F
:1065F000B0C5C9FFFF0E9EB602D0E82EFCD79E960E
:10660000C69EB1C5C9FFFF0E9EB602D0E82EFCD7CC
:106610009E96C69EB2C5C9FFFF0E9EB602D0E82E5A
:10662000FCD79E96C69EB3C5C9FFFF0E9EB602D08C
:10663000E82EFCD79E96C69EB4C5C9FFFF0E9EB637
:1066400002D0E82EFCD79E96C69EB5C5C9FFFF0EA8
:106650009EB602D0E82EFCD752EC32F012003BEC92
:1066600032F000012550FD0AD8B442EF33F09E9677
:10667000C69E070EC96EFF0E9EB602D0E82EFCD74E
:106680004BEF33F09E96C69E090EC96EFF0E9EB666
:1066900002D0E82EFCD79E96C69E000EC96EFF0E55
:1066A0009EB602D0E82EFCD7C9CFAFF59E96C69E07
:1066B000000EC96EFF0E9EB602D0E82EFCD7C9CFE1
:1066C000B0F59E96C69E000EC96EFF0E9EB602D015
:1066D000E82EFCD7C9CFB1F59E96C69E000EC96EB6
:1066E000FF0E9EB602D0E82EFCD7C9CFB2F552EC11
:1066F00032F03BEC32F09E96C69E26C0C9FFFF0EDC
:106700009EB602D0E82EFCD79E96C69E000EC96E9D
:10671000FF0E9EB602D0E82EFCD7C9CFB6F552ECDC
:1067200032F012003BEC32F000012550FD0AD8B4E3
:10673000A5EF33F09E96C69E870EC96EFF0E9EB6DD
:1067400002D0E82EFCD7AEEF33F09E96C69E890E9F
:10675000C96EFF0E9EB602D0E82EFCD79E96C69E4E
:10676000000EC96EFF0E9EB602D0E82EFCD79E9694
:10677000C69E800EC96EFF0E9EB602D0E82EFCD7D4
:106780009E96C69E800EC96EFF0E9EB602D0E82E63
:10679000FCD79E96C69E800EC96EFF0E9EB602D096
:1067A000E82EFCD752EC32F0120000012550FE0A10
:1067B000D8B4E4EF33F000012550FD0AD8B4FBEF64
:1067C00033F02FEC33F012003BEC32F09E96C69E75
:1067D0008F0EC96EFF0E9EB602D0E82EFCD79E9695
:1067E000C69E000EC96EFF0E9EB602D0E82EFCD7E4
:1067F00052EC32F012003BEC32F09E96C69E8E0EAA
:10680000C96EFF0E9EB602D0E82EFCD79E96C69E9D
:10681000000EC96EFF0E9EB602D0E82EFCD752ECD9
:1068200032F0120000012550FE0AD8B44BEF34F0CC
:1068300000012550FD0AD8B478EF34F03BEC32F07B
:106840009E96C69E27C0C9FFFF0E9EB602D0E82EB8
:10685000FCD79E96C69E010EC96EFF0E9EB602D054
:10686000E82EFCD752EC32F03BEC32F09E96C69EFE
:10687000910EC96EFF0E9EB602D0E82EFCD79E96F2
:10688000C69EA50EC96EFF0E9EB602D0E82EFCD79E
:1068900052EC32F012003BEC32F09E96C69E27C0BE
:1068A000C9FFFF0E9EB602D0E82EFCD79E96C69E6C
:1068B000450EC96EFF0E9EB602D0E82EFCD752ECF4
:1068C00032F03BEC32F09E96C69E8F0EC96EFF0EE4
:1068D0009EB602D0E82EFCD79E96C69E000EC96ECC
:1068E000FF0E9EB602D0E82EFCD752EC32F012001A
:1068F0003BEC32F09E96C69E27C0C9FFFF0E9EB6A7
:1069000002D0E82EFCD79E96C69E3D0EC96EFF0EA5
:106910009EB602D0E82EFCD752EC32F03BEC32F0BF
:106920009E96C69E8F0EC96EFF0E9EB602D0E82EB2
:10693000FCD79E96C69EA90EC96EFF0E9EB602D0CB
:10694000E82EFCD752EC32F012003BEC32F09E966F
:10695000C69E27C0C9FFFF0E9EB602D0E82EFCD708
:106960009E96C69E810EC96EFF0E9EB602D0E82E80
:10697000FCD752EC32F012003BEC32F09E96C69EF1
:1069800027C0C9FFFF0E9EB602D0E82EFCD79E9608
:10699000C69E010EC96EFF0E9EB602D0E82EFCD731
:1069A00052EC32F012003BEC32F09E96C69E910EF5
:1069B000C96EFF0E9EB602D0E82EFCD79E96C69EEC
:1069C000A50EC96EFF0E9EB602D0E82EFCD752EC83
:1069D00032F012003BEC32F09E96C69E910EC96ECC
:1069E000FF0E9EB602D0E82EFCD79E96C69E000EE5
:1069F000C96EFF0E9EB602D0E82EFCD752EC32F0E4
:106A000012000501256B266B276B286B899A400EB7
:106A1000C76E200EC66E9E96C69E030EC96EFF0EF2
:106A20009EB602D0E82EFCD79E96C69E27C5C9FF0B
:106A3000FF0E9EB602D0E82EFCD79E96C69E26C5B7
:106A4000C9FFFF0E9EB602D0E82EFCD79E96C69ECA
:106A500025C5C9FFFF0E9EB602D0E82EFCD79E9634
:106A6000C69EC952FF0E9EB602D0E82EFCD7898A78
:106A70000F01C950FF0A01E1120005012E51130A4E
:106A800005E005012E51170A0CE012000501F00E79
:106A9000256FFF0E266F0F0E276F000E286F5AEF1F
:106AA00035F00501F00E256FFF0E266FFF0E276FE4
:106AB000000E286F899A400EC76E200EC66E9E96F5
:106AC000C69E030EC96EFF0E9EB602D0E82EFCD7FE
:106AD0009E96C69E27C5C9FFFF0E9EB602D0E82E21
:106AE000FCD79E96C69E26C5C9FFFF0E9EB602D055
:106AF000E82EFCD79E96C69E25C5C9FFFF0E9EB602
:106B000002D0E82EFCD79E96C69EC952FF0E9EB6B6
:106B100002D0E82EFCD7898A0F01C950FF0A1DE078
:106B200005012E51130A05E005012E51170A0BE04D
:106B300012000501000E256F000E266F100E276F44
:106B4000000E286F12000501000E256F000E266F43
:106B5000000E276F010E286F12000501256B266BB2
:106B6000276B286B05012E51130A05E005012E51F4
:106B7000170A0CE012000501000E216F000E226FB3
:106B8000080E236F000E246FCFEF35F00501000EC5
:106B9000216F000E226F800E236F000E246F21C51F
:106BA00000F122C501F123C502F124C503F125C579
:106BB00004F126C505F127C506F128C507F1F0EC5B
:106BC0002EF000C125F501C126F502C127F503C14C
:106BD00028F5899A400EC76E200EC66E9E96C69EF8
:106BE000030EC96EFF0E9EB602D0E82EFCD79E960D
:106BF000C69E27C5C9FFFF0E9EB602D0E82EFCD761
:106C00009E96C69E26C5C9FFFF0E9EB602D0E82EF0
:106C1000FCD79E96C69E25C5C9FFFF0E9EB602D024
:106C2000E82EFCD79E96C69EC952FF0E9EB602D095
:106C3000E82EFCD7898AC950FF0A08E104C125F56E
:106C400005C126F506C127F507C128F5D89005012D
:106C500024332333223321332151F00B216F0501DB
:106C600021673AEF36F022673AEF36F023673AEFC2
:106C700036F02467CFEF35F00501100E2527E86ABE
:106C80002623E86A2723E86A28231200E86A050118
:106C90002E51130A06E005012E51170A0BE0020ED1
:106CA000120005012851000A03E12751F00B07E00B
:106CB000010E120005012851000A01E0010E120028
:106CC00029C500F12AC501F12BC502F12CC503F13C
:106CD00025C504F126C505F127C506F128C507F12C
:106CE0009FEC30F003BF120046EC36F0D8A4D8EF8A
:106CF00036F0899A400EC76E200EC66E9E96C69ECE
:106D0000060EC96EFF0E9EB602D0E82EFCD7898A09
:106D1000899A9E96C69E020EC96EFF0E9EB602D03E
:106D2000E82EFCD79E96C69E27C5C9FFFF0E9EB6CD
:106D300002D0E82EFCD79E96C69E26C5C9FFFF0E40
:106D40009EB602D0E82EFCD79E96C69E25C5C9FFEA
:106D5000FF0E9EB602D0E82EFCD79E96C69E000E71
:106D6000C96EFF0E9EB602D0E82EFCD7898A899A9A
:106D70009E96C69E050EC96EFF0E9EB602D0E82EE8
:106D8000FCD79E96C69EC952FF0E9EB602D0E82E34
:106D9000FCD7C9B0C1EF36F0898A0501100E25274E
:106DA000E86A2623E86A2723E86A282360EF36F09A
:106DB0001200899A400EC76E200EC66E9E96C69E21
:106DC000060EC96EFF0E9EB602D0E82EFCD7898A49
:106DD000899A9E96C69EC70EC96EFF0E9EB602D0B9
:106DE000E82EFCD7898A0501256B266B276B286B5B
:106DF0001200899A400EC76E200EC66E9E96C69EE1
:106E0000050EC96EFF0E9EB602D0E82EFCD79E96E8
:106E1000C69EC952FF0E9EB602D0E82EFCD7C9CF3F
:106E200037F5898A1200899A400EC76E200EC66E09
:106E30009E96C69EB90EC96EFF0E9EB602D0E82E73
:106E4000FCD7898A1200899A400EC76E200EC66E42
:106E50009E96C69EAB0EC96EFF0E9EB602D0E82E61
:106E6000FCD7898AFF0EE82EFED7120046EC36F0DA
:106E7000D8A41200899A400EC76E200EC66E9E9648
:106E8000C69E030EC96EFF0E9EB602D0E82EFCD73A
:106E90009E96C69E27C5C9FFFF0E9EB602D0E82E5D
:106EA000FCD79E96C69E26C5C9FFFF0E9EB602D091
:106EB000E82EFCD79E96C69E25C5C9FFFF0E9EB63E
:106EC00002D0E82EFCD79E96C69EC952FF0E9EB6F3
:106ED00002D0E82EFCD7898A0F01C950FF0AD8A436
:106EE000B5EF38F00501FE0E376F0501FF0E536F49
:106EF000FF0E546FFF0E556FFF0E566F15A6379994
:106F0000158665EC32F0AFC538F5B0C539F5B1C5B9
:106F10003AF5B2C53BF5B3C53CF5B4C53DF5B5C5CD
:106F20003EF50784BAC166F1BBC167F1BCC168F127
:106F3000BDC169F14BC14FF14CC150F14DC151F18F
:106F40004EC152F157C159F158C15AF100011650C2
:106F5000010AD8B4BAEF37F000011650020AD8B4CB
:106F6000DFEF37F000011650040AD8B404EF38F010
:106F7000B5EF38F00501476B486B496B4A6B05016B
:106F80004B6B4C6B4D6B4E6B05014F6B506B516BEC
:106F9000526B8BA0379B8EEC22F000C1DAF101C15D
:106FA000DBF102C1DCF103C1DDF100C13FF501C13C
:106FB00040F502C141F503C142F523EF38F0050168
:106FC000476B486B496B4A6B05014B6B4C6B4D6BC8
:106FD0004E6B05014F6B506B516B526B8EEC22F078
:106FE00000C1DAF101C1DBF102C1DCF103C1DDF165
:106FF0008BEC23F000C147F501C148F502C149F50A
:1070000003C14AF5B5EF38F0379BDAC13FF5DBC174
:1070100040F5DCC141F5DDC142F58EEC22F000C146
:107020004BF501C14CF502C14DF503C14EF58BEC9A
:1070300023F000C14FF501C150F502C151F503C164
:1070400052F523EF38F0050161672EEF38F06267E3
:107050002EEF38F063672EEF38F0646732EF38F0C8
:1070600047EF38F0DAC100F1DBC101F1DCC102F118
:10707000DDC103F161C504F162C505F163C506F127
:1070800064C507F19FEC30F003BFB5EF38F059C18C
:1070900043F55AC144F5B9C545F50501110E326FE6
:1070A000899A400EC76E200EC66E9E96C69E060E2C
:1070B000C96EFF0E9EB602D0E82EFCD7898A899A47
:1070C0009E96C69E020EC96EFF0E9EB602D0E82E98
:1070D000FCD79E96C69E27C5C9FFFF0E9EB602D05E
:1070E000E82EFCD79E96C69E26C5C9FFFF0E9EB60B
:1070F00002D0E82EFCD79E96C69E25C5C9FFFF0E7E
:107100009EB602D0E82EFCD725EE37F0322F02D003
:1071100095EF38F09E96C69EDECFC9FFFF0E9EB655
:1071200002D0E82EFCD786EF38F0898A899A9E969D
:10713000C69E050EC96EFF0E9EB602D0E82EFCD785
:107140009E96C69EC952FF0E9EB602D0E82EFCD770
:10715000C9B0A0EF38F0898A0501100E2527E86A2A
:107160002623E86A2723E86A28231590079412004B
:1071700021C500F122C501F123C502F124C503F1A7
:10718000899A400EC76E200EC66E9E96C69E0B0E46
:10719000C96EFF0E9EB602D0E82EFCD79E96C69E04
:1071A00002C1C9FFFF0E9EB602D0E82EFCD79E9604
:1071B000C69E01C1C9FFFF0E9EB602D0E82EFCD7C5
:1071C0009E96C69E00C1C9FFFF0E9EB602D0E82E55
:1071D000FCD79E96C69EC952FF0E9EB602D0E82EE0
:1071E000FCD725EE37F00501100E326F9E96C69E35
:1071F000C952FF0E9EB602D0E82EFCD7C9CFDEFFE3
:10720000322FF6EF38F0898A1200899A400EC76E45
:10721000200EC66E9E96C69E900EC96EFF0E9EB63E
:1072200002D0E82EFCD79E96C69E000EC96EFF0EB9
:107230009EB602D0E82EFCD79E96C69E000EC96E62
:10724000FF0E9EB602D0E82EFCD79E96C69E000E7C
:10725000C96EFF0E9EB602D0E82EFCD79E96C69E43
:10726000C952FF0E9EB602D0E82EFCD7C9CF2DF52D
:107270009E96C69EC952FF0E9EB602D0E82EFCD73F
:10728000C9CF2EF5898A120065EC32F005012F5125
:10729000010A61E005012F51020A16E005012F5194
:1072A000030A1BE005012F51040A26E005012F51B6
:1072B000050A2DE005012F51060A3BE005012F517B
:1072C000070A41E0ABEF39F015B01200602FA9EFCB
:1072D00039F05FC560F5ABEF39F0B0C500F10101E1
:1072E0000F0E001701010051000A35E001010051A5
:1072F000050A31E0A9EF39F0B0C500F101010F0E28
:10730000001701010051000A26E0A9EF39F005013C
:10731000B051000A20E00501B051150A1CE005013A
:10732000B051300A18E00501B051450A14E0A9EF48
:1073300039F00501B051000A0EE00501B051300AE4
:107340000AE0A9EF39F00501B051000A04E0A9EF05
:1073500039F015901200158012008B906BEC2FF015
:10736000B9C5E8FFD70802E36BEC2FF0B9C5E8FF19
:10737000C80802E36BEC2FF0B9C5E8FFB90802E3D7
:107380006BEC2FF0B9C5E8FFAA0802E36BEC2FF015
:10739000B9C5E8FF9B0802E36BEC2FF013EC37F064
:1073A000F29CF29E8B94C69AC2909482948C720E38
:1073B000D36ED3A4FED789968A909390F29AF294D2
:1073C0009D909E909D929E92F298F292D5EC33F011
:1073D000FF0EE8CF00F0E82EFED7002EFCD7F2908B
:1073E000F2868150FF0EE82EFED7F29081A8FBEFC7
:1073F00039F0F29E0300700ED36EF296F29015846F
:0A74000003808CEC2FF09AEF0BF0E4
:10BF0000E844F926000C160C2B0C3F0C520C640C68
:10BF1000760C860C960CA50CB30CC10CCF0CDC0C6B
:06BF2000E80CF40C000C1B
:0200000400F00A
:0100C800FD3A
:00000001FF
